:100000000C94C8000C94E4340C94D30D0C94E500CB
:100010000C94E5000C94E5000C94E5000C94E500CC
:100020000C94E5000C94E5000C94E5000C943B1056
:100030000C94E5000C94732E0C94AD2E0C94D62EDB
:100040000C94E5000C94E5000C94E5000C94B1369A
:100050000C94E50031313056332E33370000000167
:100060000000060000FF00000F02000C0014010158
:100070000400001450040100000000000000000013
:1000800000000000010003E8000000000000000381
:10009000E800000000000200FA0600070000FF0070
:1000A0000037060002800000000000002107101049
:1000B0000504030206100D0C0B0A2E1005040302A2
:1000C00006100D0C0B0A2E100504030206100D0C71
:1000D0000B0A2E1111111111111111111111111100
:1000E0001111111111111111111111111111110011
:1000F0000404040808080C0C0C1010101414181830
:10010000181C1C1C20202020242424282828282CCB
:100110002C2C2C30303030343434343438383838B7
:10012000383838383C3C3C3C3C3C3C3C3C3C3C1843
:10013000180B0B0C0C0B0C0B040208040C1803031B
:10014000030801010101010804040101000000008D
:1001500000000C10140808090A0B0C08080C090A06
:100160000B0C0D0E080808090A0A0A0A0A0B0C0CE7
:1001700000010405030647401D1B1C1B14133322FA
:1001800019100C080603016744332219100C0803E8
:1001900011241FBECFE5D8E0DEBFCDBF11E0A0E641
:1001A000B0E0EAE0F3E702C005900D92A431B10798
:1001B000D9F716E0A4E1B1E001C01D92A037B10764
:1001C000E1F70E94E7000C9484390C940000EF9250
:1001D000FF920F931F93CF93DF93CDB7DEB7249792
:1001E0000FB6F894DEBF0FBECDBF0E94960E82E020
:1001F0000E9414100E940A0F8DB18F738DB981E88F
:1002000087BB30E020E018BA00000000000096B381
:1002100080E888BB000000000000B69B02C096FF8B
:100220002F5F3F5F3A3079F72A3039F560E089E097
:1002300090E00E94810F60E080E090E00E94810FDA
:100240001A82198205C089819A8101969A838983CD
:1002500089819A818F5F9F4FB1F7C0981A82198266
:1002600005C089819A8101969A83898389819A81BF
:100270008F5F9F4FB1F7C09AE3CF0E94960E82E046
:100280000E9414100E94E50D0E9496100E940A0F11
:10029000AB980E94D70E0E94ED0E80E090E00E9485
:1002A000790F843E09F4DBC0C0980E94922F60E071
:1002B00089E090E00E94810F40E16DE570E080E010
:1002C00090E00E94C60F61E08AE491E00E94810FF5
:1002D00060E08BE491E00E94810F60E08CE491E0AB
:1002E0000E94810F60E08DE491E00E94810F62E046
:1002F0008EE491E00E94810F60E08FE491E00E9423
:10030000810F60E080E591E00E94810F60E081E56F
:1003100091E00E94810F0E949E0F4DE26CE770E019
:100320008DE390E00E94C60F4DE26CE770E08AE634
:1003300090E00E94C60F4DE26CE770E087E990E024
:100340000E94C60F43E069EA70E084EC90E00E94EE
:10035000C60F43E06CEA70E087EC90E00E94C60FA5
:1003600040E86FEA70E08AEC90E00E94C60F64E615
:100370008AE591E00E94810F60E08BE591E00E94A8
:10038000810F64E68CE591E00E94810F60E08DE5CD
:1003900091E00E94810F64E68EE591E00E94810F5A
:1003A00060E08FE591E00E94810F60E080E691E0DF
:1003B0000E94810F60E081E691E00E94810F60E081
:1003C00082E691E00E94810F60E083E691E00E9466
:1003D000810F60E084E691E00E94810F60E085E695
:1003E00091E00E94810F60E08DEF93E00E94810F09
:1003F00060E08EEF93E00E94810F60E08FEF93E06A
:100400000E94810F60E086E691E00E94810F68E023
:1004100087E691E00E94810F60E088E691E00E940B
:10042000810F68E089E691E00E94810F60E08AE632
:1004300091E00E94810F68E08BE691E00E94810FBD
:1004400081E090E00E94790FEEE5F0E0E4918E17F4
:1004500029F464EE80E090E00E94810FC09A81E070
:1004600090E00E94790F0E94EB2E8AE090E00E94BB
:10047000790F8093C104882311F00E94B5378EE76D
:100480000E94B60A00E0802F80610E94B60A802F89
:1004900088610E94B60A802F84600E94B60A802F6D
:1004A00086600E94B60A802F84610E94B60A005EB0
:1004B000003649F70E9435090E94EE0FEE24FF2412
:1004C000C70125E0880F991F2A95E1F78D600E94EA
:1004D0004B0F082F10E0C80101960E94790F8C8302
:1004E000C80102960E94790F8B836B817C818E2DCF
:1004F0000E94F107C70185960E94790F682F8E2D03
:100500000E94480F0894E11CF11C83E0E816F104F6
:10051000B9F62FEF4FEF60E086E10E9451052FEF13
:100520004FEF60E086E30E9451052FEF4FEF60E050
:1005300086E50E9451058AE491E00E94790F80933C
:100540002F068BE491E00E94790F809330068CE4B3
:1005500091E00E94790F809331068DE491E00E9432
:10056000790F809332068EE491E00E94790F809398
:10057000E7058FE491E00E94790F8093E80580E51C
:1005800091E00E94790F8093E90581E591E00E9456
:10059000790F8093EA05E0902F06F09030060091E5
:1005A00031061091320685E090E00E94790FB80183
:1005B000A70190E00E94DD338AE591E00E94790F67
:1005C000809310068BE591E00E94790F80931106CD
:1005D0008CE591E00E94790F809312068DE591E001
:1005E0000E94790F809313068EE591E00E94790FA7
:1005F000809314068FE591E00E94790F8093150691
:1006000080E691E00E94790F8093F20581E691E007
:100610000E94790F8093F30582E691E00E94790FA2
:100620008093F40583E691E00E94790F8093F505AD
:1006300084E691E00E94790F8093F60585E691E0CB
:100640000E94790F8093F7058DEF93E00E94790F58
:10065000809317068EEF93E00E94790F809318061F
:100660008FEF93E00E94790F8093190686E691E060
:100670000E94790F80935B0187E691E00E94790FD9
:1006800080935C0188E691E00E94790F80935D0180
:1006900089E691E00E94790F80935E018AE691E0FD
:1006A0000E94790F80935F018BE691E00E94790FA1
:1006B0008093600182E090E00E94790F0E94723680
:1006C0000E94F22D0E94700378940E940F060E94EF
:1006D0009C100E94EC0A0E94B6280E947603F5CF77
:1006E00081E08093CF041092B00508958091330685
:1006F00081FF07C08091B0058F3F19F08F5F809315
:10070000B0058091CF04813051F48091B0058F30D5
:1007100030F0C0981092B00582E08093CF048091B1
:10072000CF04823051F48091B005853030F0C09A0A
:100730001092B00581E08093CF0408950895089544
:1007400008950895089508950895CF92DF92FF9235
:100750000F931F93CF93DF93CDB7DEB729970FB6D3
:10076000F894DEBF0FBECDBF82E00E94C3108CE0C4
:1007700090E00E94790F898382E090E00E94790FD7
:100780008A8381E88B8381E48C838091CC058D837F
:100790008091CB058E838091CD058F838091CF058D
:1007A000888719868E010F5F1F4F89E0C82ED12CD4
:1007B000CC0EDD1EF801F0808985F80EF986809157
:1007C0006201882319F480810E94372F0F5F1F4F29
:1007D0000C151D0579F780916201882319F48F2D7E
:1007E0000E94372F29960FB6F894DEBF0FBECDBFFB
:1007F000DF91CF911F910F91FF90DF90CF900895DF
:10080000682F70E080FD2FC0CB018076907035E0BE
:10081000959587953A95E1F7E82FCB018F79907000
:100820008431910529F4F0E0E45DF94F20830895C7
:100830008630910541F4F0E0EE0FFF1FEB52FA4FC6
:10084000208341830895089771F4F0E0EE0FFF1FB5
:10085000EA5DF94F2083418343FF05C08081918188
:10086000906F918380830895EF92FF920F931F936F
:10087000182F062FF42EE22E0E9400048BB78F7BD8
:100880008BBFC398812F0E942310802F0E942310BA
:100890008F2D0E9423108E2D0E942310C39A8BB798
:1008A00080648BBF1F910F91FF90EF900895CF92BE
:1008B000DF92EF92FF920F931F93CF93DF937C0110
:1008C0006B01DC018C9190E09C012F793070211537
:1008D000310519F02830310501F5EC01C076D070F2
:1008E00045E0D595C7954A95E1F7C330B0F48C2F14
:1008F0008B5E0E940010682F8C2F0E94480FEC2FF7
:10090000F0E09F0129533A4FDF01A05ABF4F8C916D
:10091000D9018C93E650FA4F1082F701238142816E
:10092000618180810E9400048BB78F7B8BBFC3984D
:10093000C0E0D0E086010C0F1D1FF701EC0FFD1F7A
:1009400080810E942310D8018C932196C430D10558
:1009500089F7C39A8BB780648BBF80E090E0DF910A
:10096000CF911F910F91FF90EF90DF90CF9008955E
:100970005F926F927F928F929F92AF92BF92CF922F
:10098000DF92EF92FF920F931F93CF93DF93CDB738
:10099000DEB728970FB6F894DEBF0FBECDBF282F65
:1009A00030E0F901EC53FA4F8081882319F4662373
:1009B00009F461C060831A82C901880F991F820FF0
:1009C000931F880F991F880F991FF0E85F2E580E0C
:1009D00000E010E0862F90E0E4E0AE2EB12CA822DB
:1009E000B92272E0C72ED12CC822D92261E0E62EAE
:1009F000F12CE822F92255E0652E712C6C0E7D1E3B
:100A00004E010894811C911CA114B10489F0063098
:100A100020F4E114F10421F006C0C114D10419F44A
:100A200090E180E102C091E181E18B839C830CC065
:100A3000C80185539F4F0E94790F8B83C80186534D
:100A40009F4F0E94790F8C83902F002311F0063066
:100A500011F480E18C839A3019F48B8180628B834E
:100A6000950D9983B301C4010E9457040E5F1F4F77
:100A70000C30110549F628960FB6F894DEBF0FBE6C
:100A8000CDBFDF91CF911F910F91FF90EF90DF903D
:100A9000CF90BF90AF909F908F907F906F905F901E
:100AA00008953F924F925F926F927F928F929F92A2
:100AB000AF92BF92CF92DF92EF92FF920F931F936C
:100AC000CF93DF93CDB7DEB728970FB6F894DEBF8C
:100AD0000FBECDBFC82E562E442E322E90E09C0164
:100AE0002F7930702115310521F02830310509F0BA
:100AF00064C08076907045E0959587954A95E1F7BA
:100B0000D82E82E08D1508F458C0ED2CFF24F70193
:100B1000EE0FFF1FDF01AE50BA4F8D919C91EE5A40
:100B2000FE4F91838083F701E85AFE4F808188232E
:100B300071F110821A828CE0D89EC00111248C01C0
:100B400000581F4F2CE8A22EB12CA80EB91E85E02C
:100B5000682E712C6C0E7D1E4E010894811C911C18
:100B600013C00983C801855B9F4F0E94790F8B8357
:100B7000C801865B9F4F0E94790F8C83B301C4012B
:100B80000E9457040E5F1F4F0A151B0550F38D2D51
:100B90008B5E0E940010682F8D2D0E94480FD70198
:100BA000A953BA4FF701E05AFF4F80818C93EAEFC7
:100BB000F5E0EE0EFF1EF7011082232D442D652D6A
:100BC0008C2D0E9400048BB78F7B8BBFC3988C2D1C
:100BD0000E942310852D0E942310842D0E94231033
:100BE000832D0E942310C39A8BB780648BBF2896F5
:100BF0000FB6F894DEBF0FBECDBFDF91CF911F912E
:100C00000F91FF90EF90DF90CF90BF90AF909F90AB
:100C10008F907F906F905F904F903F900895AF922C
:100C2000BF92CF92DF92EF92FF920F931F93CF93D9
:100C3000DF93CDB7DEB72A970FB6F894DEBF0FBEAD
:100C4000CDBF1092B9051092BA051092BB058091E4
:100C5000C205882311F083995FC0809114018F5FD2
:100C600080931401833010F0109214018EE090E014
:100C70000E94790F8F5F8093C20580911401829545
:100C8000880F807E8B608F838E010D5F1F4F67E022
:100C9000C62ED12CCC0EDD1EB801C6010E94570411
:100CA0008B818093C3058D8183FF02C0806F8D830C
:100CB0008D818A838E818983E0911401F0E0EE0FAB
:100CC000FF1FE454FA4F89819A819183808383992D
:100CD00023C0EE24FF2458011E2D1295110F107E03
:100CE000812F87618F83B501C6010E945704F701E8
:100CF000E754FA4F8E81808316611F838FEF8987B7
:100D00008A87B501C6010E9457040894E11CF11CB2
:100D100083E0E816F10401F72A960FB6F894DEBFD7
:100D20000FBECDBFDF91CF911F910F91FF90EF903C
:100D3000DF90CF90BF90AF900895CF93DF93EC01F9
:100D400082E090E00E94790F809328019091250124
:100D5000992359F08091330680FF03C091509093FE
:100D600025018091240181600EC080912701882394
:100D700039F0809124018061809324011092270131
:100D8000809124018E7F8093240180912701882304
:100D9000F1F585E191E00E940C338823C1F12091A7
:100DA00018013091190140911A0150911B01809155
:100DB0002F0690913006A0913106B0913206281787
:100DC00039074A075B0719F580911501873008F448
:100DD00080C09E01295F3F4F809128018F83ECE105
:100DE000F1E0DE0180818D93E90188819191890F85
:100DF000888381E0E332F807A9F7809115018730F5
:100E000011F481E001C082E08093DF056DC0809124
:100E10002701882379F468E0CE010E947E3688237A
:100E200049F08F8190912801890F8F8381E0809311
:100E300016065AC00E94132F8F3F31F4809124016F
:100E40008061809324013AC089E291E00E94532F8F
:100E50008130A1F584E1809325012091270122238F
:100E600029F4809129018093260125C090912601C3
:100E7000809128019817D1F430912401932F946028
:100E80009093240191FD12C0C20FD11D2197809132
:100E900029018883283051F494FF04C09F7E9093E9
:100EA000240106C036603093240102C0283018F0B7
:100EB0001092270103C02F5F209327011092DF05B6
:100EC000109216068091240184FF06C08F7E8093C5
:100ED00024018FEF9FEF0AC081FD03C080E090E006
:100EE00005C08D7F8093240181E090E0DF91CF9158
:100EF0000895FB0120813181280F391F35952795F1
:100F000031832083C9010895FF920F931F93F62E1A
:100F100081608093DB0500EE15E0B8018BED95E074
:100F20000E9457040F0D111DF801808190E01F9160
:100F30000F91FF90089581608093DB0560EE75E06E
:100F40008BED95E00E9457048091E30590E00895B1
:100F500081608093DB0560EE75E08BED95E00E948B
:100F600057042091E20530E0522F44278091E30599
:100F700090E0482B592B23FD02C0CA010895CA01F5
:100F8000906F0895CF93DF93CDB7DEB724970FB658
:100F9000F894DEBF0FBECDBF81608093DB0560EEAD
:100FA00075E08BED95E00E9457049091E10597FF65
:100FB00003C08FEF8C8301C01C829B838091E2056C
:100FC0008A838091E305898369817A818B819C8101
:100FD00024960FB6F894DEBF0FBECDBFDF91CF9140
:100FE0000895CF92DF92FF920F931F93CF93DF93D9
:100FF000CDB7DEB721970FB6F894DEBF0FBECDBFD9
:101000008B01F82EF294FF0C70EEF7228F2D896180
:101010008093DB0560EE75E08BED95E00E94570450
:10102000C8018070987F892B19F08FEF9FEF57C010
:101030008091E205982F9F709C5F82958F70981B1E
:101040000F3F1105F9F0F4F06801191694F0412FE3
:101050005527202F60E08F2D8C600E94510520E0E5
:101060004FE760E08F2D82610E94510581E090E0A2
:1010700036C0D594C79491508FEFC816D104E1F0D3
:10108000DCF0E3CF68019D3094F0412F5527202FED
:1010900060E08F2D8C600E9451052DE040E060E003
:1010A0008F2D82610E94510582E090E018C0CC0C27
:1010B000DD1C9F5FC7FEE7CF412F5527202F60E043
:1010C0008F2D8C6099830E9451059981292F4C2D79
:1010D00060E08F2D82610E94510580E090E02196B2
:1010E0000FB6F894DEBF0FBECDBFDF91CF911F9139
:1010F0000F91FF90DF90CF9008950F931F93062FCD
:10110000182F1295110F107E812F85618093DB05BA
:1011100060EE75E08BED95E00E945704202F409122
:10112000E20560E0812F84610E9451051F910F91BB
:101130000895CF93DF93CDB7DEB724970FB6F89419
:10114000DEBF0FBECDBF49835A836B837C83298169
:101150004A816B810E94510524960FB6F894DEBF38
:101160000FBECDBFDF91CF9108951F93182F62E07E
:101170000E947D081295110F107E40E050E060E063
:1011800070E0812F88600E94990840E050E060E0A4
:1011900070E0812F8A600E9499081F9108958295BE
:1011A000880F807E40E050E060E070E088600E9440
:1011B00099080895E82FF0E0EE0FFF1FE35AF94F6A
:1011C00040815181662329F002C0559547956A9563
:1011D000E2F7509541955F4F662757FD6095762F52
:1011E0008295880F807E88600E9499080895E82F74
:1011F000F0E0EE0FFF1FE35AF94F40815181662363
:1012000029F002C0559547956A95E2F7662757FD84
:101210006095762F8295880F807E88600E9499085D
:1012200008950F931F93CF93DF93CDB7DEB7229727
:101230000FB6F894DEBF0FBECDBF8C0101970E94A0
:10124000790FFE0131968183C8010E94790F89834D
:1012500089819A8122960FB6F894DEBF0FBECDBF6A
:10126000DF91CF911F910F910895CF92DF92EF926E
:10127000FF920F931F93CF93DF93CDB7DEB72897DD
:101280000FB6F894DEBF0FBECDBF1A820BEC10E094
:1012900085E0C82ED12CCC0EDD1E7E010894E11C09
:1012A000F11C802F8B548983C8010E94790F8B8396
:1012B000C80101970E94790F8C83B601C7010E9473
:1012C00057040E5F1F4F81E00B34180751F7289623
:1012D0000FB6F894DEBF0FBECDBFDF91CF911F9147
:1012E0000F91FF90EF90DF90CF9008951F93909112
:1012F000300180912F01981719F480E090E040C0F0
:10130000E92FF0E0EB5BFE4F1081892F8F5F809318
:1013100030018A3011F410923001EDE1F6E01192C3
:1013200086E0E632F807D9F78CE090E00E94790F6A
:1013300080931D0682E090E00E94790F80931E0644
:1013400080E880931F068AE8809320061093240685
:1013500020911B06233019F4EEE1F6E005C08091E0
:101360001D0680932506F8CF819190912506890F5F
:101370008093250686E0E532F807B1F7822F90E0EA
:101380001F910895EF92FF920F931F938B01E82E08
:10139000FF24C70125E0880F991F2A95E1F788618E
:1013A0000E949B07877002C0000F111F8A95E2F709
:1013B000612F772767FD7A95C7014C960E94810FB0
:1013C000602FC7014F960E94810F1F910F91FF90D0
:1013D000EF900895CF92DF92EF92FF920F931F93B9
:1013E000CF93DF93CDB7DEB728970FB6F894DEBF63
:1013F0000FBECDBF1A820BE011E035E0C32ED12C19
:10140000CC0EDD1E7E010894E11CF11C802F8A5455
:101410008983B601C7010E9457046F81C8010E94E9
:10142000810F6885C80101970E94810F0E5F1F4FD1
:1014300081E00B34180751F728960FB6F894DEBFF9
:101440000FBECDBFDF91CF911F910F91FF90EF9015
:10145000DF90CF900895CF92DF92EF92FF920F939B
:101460001F93CF93DF93CDB7DEB728970FB6F894CD
:10147000DEBF0FBECDBF1A820BEC10E045E0C42EDC
:10148000D12CCC0EDD1E7E010894E11CF11C802FB6
:101490008A548983B601C7010E9457046F81C8012D
:1014A0000E94810F6885C80101970E94810F0E5F1D
:1014B0001F4F81E00B34180751F728960FB6F894A8
:1014C000DEBF0FBECDBFDF91CF911F910F91FF9077
:1014D000EF90DF90CF9008950F931F93CF93DF93FA
:1014E000082F816007FD24C08093DB0560EE75E066
:1014F0008BED95E00E945704802F0E944B0FC0EEA9
:10150000D5E0002711270C1B1D0B080F111D698149
:10151000C8018C0F9D1F0E94810F823019F482E058
:1015200090E01FC0219685E0C33ED80781F717C021
:101530008093DB0560EE75E08BED95E00E9457042B
:1015400010E06091E205C801855B9F4F0E94810F0A
:101550006091E305C801865B9F4F0E94810F80E088
:1015600090E0DF91CF911F910F910895FF920F931B
:101570001F93CF93DF93CDB7DEB728970FB6F894BC
:10158000DEBF0FBECDBFF82E0E944B0F082F10E01C
:10159000F982C8010E94790F8A83C80101960E94CE
:1015A000790F8B83C80102960E94790F8C83BE014C
:1015B0006B5F7F4FCE0101960E94570480E090E060
:1015C00028960FB6F894DEBF0FBECDBFDF91CF9146
:1015D0001F910F91FF9008952F923F924F925F922B
:1015E0006F927F928F929F92AF92BF92CF92DF9233
:1015F000EF92FF920F931F93CF93DF93CDB7DEB798
:1016000024970FB6F894DEBF0FBECDBF86E090E002
:101610000E94790F8A83809141018F5F80934101FD
:101620008150823010F01092410180912A0188236C
:1016300069F480E68093DB0560EE75E08BED95E064
:101640000E94570410922B0181E01BC08130E1F40D
:1016500081E68093DB0560EE75E08BED95E00E94FE
:1016600057048091E00586FD72C08091E205869561
:10167000809587708093E4058091E3058093FD0554
:1016800082E080932A0163C0823009F060C08091BB
:101690002B01A82FB0E0FD01E95EF94F908199235D
:1016A00009F450C0FD01EC51FA4F8081891708F40C
:1016B00049C015E0AA0FBB1F1A95E1F78A2F8A606F
:1016C0000E94A807BC01892B09F43FC0A0912B01FF
:1016D0004A2F50E0FA01E45DF94F8081FA01EE0FE4
:1016E000FF1F882319F0EA5DF94F02C0EB52FA4F51
:1016F00020813181CB0177FF03C0909581959F4F69
:1017000037FF03C0309521953F4F82179307E9F4C7
:10171000FA01EE5BFE4F8081823078F08A2F0E94C2
:10172000B508E0912B01F0E0DF01A650BA4F81E04F
:101730008C93EE5BFE4F108208C08F5F8083109207
:101740002A0103C0AE5BBE4F1C9210922A01809109
:10175000330680FFAFC180E00E94C73081E00E9465
:10176000C73082E00E94C7308DE78093DB0560EED2
:1017700075E08BED95E00E94570410913001E091E7
:101780002F0170916101A0E0B0E041E050E00A2E2D
:1017900002C0440F551F0A94E2F7642F842F872359
:1017A000D9F08091E00590E09D01220F331F02C027
:1017B000959587952A95E2F780FF0EC08E2F8F5F53
:1017C0008A3009F480E0811729F0F0E0EB5BFE4FEE
:1017D0004083E82F609576231196A330B105A9F6D2
:1017E000E0932F01709361018091330681FFAEC0B9
:1017F0000FE411E0E8E56E2EE1E07E2E7CE2872E1C
:1018000071E0972E60E1462E66E0562E57ECA52E2D
:1018100055E0B52E1C821B8240E8C42E36E8332EDC
:10182000DB808B819C8125E0880F991F2A95E1F749
:101830008A600E94A8077C01F5018081E114F1040F
:1018400081F0882341F48D2D8B5E0E940010682F5B
:101850008B810E94480FEB81FC81E05AFF4F808111
:101860000BC0882341F48B810E940010682F8B816C
:101870000E94480F03C08150F5018083F20120814E
:101880003181FFEF2F3F3F07A9F4F80180818230BB
:1018900009F441C021E145E060E08C2D0E94340450
:1018A00021E14DE060E0832D0E94340482E0F801E4
:1018B000808331C0C701F7FE03C0909581959F4F8B
:1018C000F80140818217930794F0413021F127E01D
:1018D00045E060E08C2D0E9434042FE04DE060E094
:1018E000832D0E94340481E0F801808310C04423DA
:1018F00091F020E145E060E08C2D0E94340420E16D
:101900004DE060E0832D0E943404F8011082F30161
:101910001082F40110828B819C8101969C838B83C1
:101920009CE0C90E390E0F5F1F4F0894611C711C9B
:101930000894811C911CE2E0F0E04E0E5F1E0894BA
:10194000A11CB11CF4EACF1609F06ACF82EF282E51
:1019500085E0382E0CE2C02E01E0D02E1BE5412E92
:1019600011E0512EB8E56B2EB1E07B2EA2E58A2E58
:10197000A1E09A2EAA24BB248AE88983C501F5E058
:10198000880F991FFA95E1F78A600E94A8077C01E9
:1019900097FF04C0F094E194F108F394F101808181
:1019A0009181892B39F1E114F10421F5F401808151
:1019B00091810097D9F4F30180818823D9F41981AA
:1019C0001A5000E020E140E160E0812F0E943404E1
:1019D0000E5F1E5F0C30B1F720E140E360E08981CB
:1019E0000E94340481E0F301808304C00197F40174
:1019F00091838083AA2009F044C0F2018081918103
:101A0000009709F4AFC0E816F90608F4ABC0F60178
:101A10008081882309F0A6C081E0808300EC10E07B
:101A20002CE24CE260E0802F0E9434040E5F1F4FD6
:101A3000F1E000301F0709F495C0F2CF892B09F5BA
:101A4000F60180818823E9F01082EAE0EE2EE1E0E1
:101A5000FE2EC7010E94790F182FC70101960E9420
:101A6000790F212F482F60E08E2D8A540E94340474
:101A700082E090E0E80EF91E9AE4E91691E0F9069A
:101A800041F70894A11CB11CE2E0F0E02E0E3F1ECD
:101A90000894C11CD11C4E0E5F1EF981F45FF983BE
:101AA0000894611C711C82E090E0880E991EFE3A39
:101AB00009F064CF8091CA058823F9F484E080930B
:101AC000CA0568E080E096E00E94F10EA7B1B0E0A0
:101AD000AA0FBB1FAF5CBE4FE7B1F0E0EE0FFF1FD8
:101AE000E050FA4F8D919C91119720813181820FA6
:101AF000931F959587958D939C9390914101E92F24
:101B0000F0E0E151FA4F8081882319F0892F0E947B
:101B1000D5309A81992311F1EA81E13019F49A992B
:101B200006C01CC0FA81F230C9F49A9917C0AB9A6A
:101B300081E080931A0600E010E062E0802F0E94AE
:101B40007D08802F0E94CF08F801E151FA4F1082E2
:101B50000F5F1F4F0330110569F0EFCFAB98109264
:101B60001A0608C0F20180819181E816F90608F48E
:101B700067CF64CF24960FB6F894DEBF0FBECDBFFB
:101B8000DF91CF911F910F91FF90EF90DF90CF9059
:101B9000BF90AF909F908F907F906F905F904F908D
:101BA0003F902F9008951F920F920FB60F9211241D
:101BB0008F9381E08093CE058F910F900FBE0F9091
:101BC0001F9018951092CE0508951F93CF93DF9321
:101BD000CDB7DEB722970FB6F894DEBF0FBECDBFEC
:101BE00023E040E060E084E10E94340423E040E030
:101BF00060E084E30E94340423E040E060E084E598
:101C00000E94340420E040E060E08AE00E94340456
:101C100020E040E060E08AE20E94340420E040E0FE
:101C200060E08AE40E94340410E002C01431A1F0A4
:101C300020E040E060E0812F0E94340420E040E09A
:101C400060E0812F80620E94340420E040E060E088
:101C5000812F80640E9434041E5F1C3138F320E021
:101C600040E060E08EE70E94340410E020E040E0B5
:101C700060E0812F80680E9434041E5F1038B1F745
:101C80002FEF47E060E08AE00E9434041A82198254
:101C900006C0000089819A8101969A83898389818F
:101CA0009A81885B9B40ACF320E040E060E08AE0F2
:101CB0000E9434048BB78F7B8BBFC39883E00E9454
:101CC000231080E00E9423108093D20580E00E94C0
:101CD00023108093D10580E00E9423108093D005CB
:101CE000C39A8BB780648BBF20E040E060E082E065
:101CF0000E9434048091D0059091D105A091D20525
:101D0000B091D305805D9740A040B04010F480E1D1
:101D100001C088E08093D40522960FB6F894DEBF08
:101D20000FBECDBFDF91CF911F910895CF93DF9369
:101D3000CDB7DEB722970FB6F894DEBF0FBECDBF8A
:101D40008EEF8ABB8CE08BBB8DEB87BB8FE188BBB2
:101D50008CEF84BB83EF85BB82EF81BB85E082BBC8
:101D6000DB981A82198206C0000089819A81019647
:101D70009A83898389819A8184369105ACF3DB9AB1
:101D80001A82198206C0000089819A8101969A837D
:101D9000898389819A8184369105ACF322960FB6A6
:101DA000F894DEBF0FBECDBFDF91CF91089581B310
:101DB000806B81BB81EF8FBD81E08EBD81E785BDEA
:101DC0000895882319F41BBC6ABD0895813019F465
:101DD00019BC68BD089563BD089517B886EC86B92F
:101DE0000895E7B1F0E0EE0FFF1FE80FF91F84B18F
:101DF00095B19183808387B190E070E0615070402D
:101E00008617970724F487B18F5F87B901C017B889
:101E1000369A08950895882309F4D99A0895882355
:101E200009F4D9980895882319F080E090E0089586
:101E300089B390E0817090700895482F662359F01F
:101E40002BB381E090E002C0880F991F4A95E2F71A
:101E5000282B2BBB08952BB381E090E002C0880FA4
:101E6000991F4A95E2F7809582238BBB08958823BA
:101E700019F080E090E008958BB390E096958795F7
:101E80008170907008958BBB089580E090E0089574
:101E90000E94E10E0895282F87FD23C0482F469504
:101EA0004F7083E0489FC001112430E020763070ED
:101EB0002115310511F4CD961AC02032310519F4DF
:101EC00086599F4F14C02034310519F489569F4F0D
:101ED0000EC04F3019F487EC90E009C04E3039F451
:101EE00004C0265B822F90E0089583E090E090E0AC
:101EF0000895DC01E199FECF0E943939802D90E0F0
:101F000008951F93CF93DF93EC01162F89E090E0A3
:101F10000E94790F882331F0C930D10519F082E091
:101F200090E008C0E199FECFDE01012E0E94413908
:101F300080E090E0DF91CF911F910895EF92FF92A2
:101F40001F93CF93DF938DE6E82E80E0F82EC0E15B
:101F5000D0E0F7011491612FCE010E94810F612F13
:101F6000CE0101960E94810F612FCE0102960E9440
:101F7000810F0894E11CF11C2396CD33D10549F75C
:101F8000DF91CF911F91FF90EF900895CF92DF9254
:101F9000EF92FF920F931F93CF93DF936C017B011E
:101FA000042F10E0C0E0D0E00CC0FE01EE0DFF1DDC
:101FB000E4916E2FCE018C0D9D1D0E94810F1F5F3D
:101FC0002196101791F780E090E0DF91CF911F915B
:101FD0000F91FF90EF90DF90CF900895CF93DF9314
:101FE000C0E1D0E0CE010E94790FFE01EC5AFE4F15
:101FF00080832196CD33D105A9F7DF91CF91089544
:10200000E4E6F1E0E80FF11D808190E008958D3263
:1020100018F081E090E00895E82FF0E0EC59FE4FD1
:10202000608380E090E0089583708DB98DB18C65F8
:102030008DB9709A1092910108958091910110923A
:10204000910190E008958FB980E009C0893C31F496
:102050008091910181608093910103C08F5F779B94
:10206000F5CF769B05C080919101826080939101AC
:102070008FB190E008951F920F920FB60F92112426
:102080008F939F93AF93BF938091D405883011F4C1
:1020900082E701C083E282BF80913406882319F071
:1020A0008150809334068091C205882319F08150B5
:1020B0008093C20580919501882321F081508093FF
:1020C00095012BC088E0809395018091920188232F
:1020D00019F08150809392018091CA05882319F0EC
:1020E00081508093CA058091EB059091EC05A091F9
:1020F000ED05B091EE050196A11DB11D8093EB0594
:102100009093EC05A093ED05B093EE058091F80552
:10211000882319F081508093F805BF91AF919F916A
:102120008F910F900FBE0F901F90189582E083BF84
:1021300081E089BF88BF0895109233068091920193
:10214000882301F59AE09093920181E08093330611
:1021500080919301882321F0815080939301089509
:102160009093930183E080933306809194018823B8
:1021700021F081508093940108959093940187E019
:102180008093330608958093C401089599E0699F70
:10219000A001112490E0837090709C01220F331FE6
:1021A000280F391F420F531F455E5D4F82E0403DAF
:1021B000580714F04BE152E0CA0108950F931F93A2
:1021C000CF93DF93CDB7DEB728970FB6F894DEBF75
:1021D0000FBECDBFE82F0D831E832F8338878093DA
:1021E0006F066093390640933A0681E080935B0660
:1021F00038853093CC052F812093CB059E81909319
:10220000CD058D818093CF059093BC018093BB0158
:102210003093C0012093BF019093BE018093BD0114
:10222000F0E0EE0FFF1FED59FF4F0190F081E02D20
:102230008091F001811109958091CC0587FF03C041
:102240008FEF8C8301C01C828091CB058B838091A2
:10225000CD058A838091CF05898369817A818B81BD
:102260009C8128960FB6F894DEBF0FBECDBFDF91DC
:10227000CF911F910F9108950000089500000895D7
:102280000000089500000895809139068823A9F47C
:102290008091420690914306A0914406B091450674
:1022A0002091BD013091BE014091BF015091C0010C
:1022B000820F931FA41FB51FC4C08130A9F4809161
:1022C000420690914306A0914406B09145062091A4
:1022D000BD013091BE014091BF015091C001821BF0
:1022E000930BA40BB50BADC0823099F460914206FC
:1022F0007091430680914406909145062091BD015E
:102300003091BE014091BF015091C0010E94B6388A
:1023100031C08330D9F460914206709143068091B8
:102320004406909145062091BD013091BE01409137
:10233000BF015091C0010E94FC38209342063093A7
:102340004306409344065093450683C08430D9F435
:102350006091420670914306809144069091450633
:102360002091BD013091BE014091BF015091C0014B
:102370000E94FC38609342067093430680934406A3
:102380009093450666C08530A9F4809142069091ED
:102390004306A0914406B09145062091BD013091BD
:1023A000BE014091BF015091C00182239323A42319
:1023B000B52347C08630A9F4809142069091430628
:1023C000A0914406B09145062091BD013091BE0117
:1023D0004091BF015091C001822B932BA42BB52BB0
:1023E00030C08730A9F48091420690914306A091B5
:1023F0004406B09145062091BD013091BE01409147
:10240000BF015091C00182279327A427B52719C087
:10241000883069F48091420690914306A091440669
:10242000B091450680959095A095B0950AC08930E9
:1024300081F48091BD019091BE01A091BF01B09146
:10244000C0018093420690934306A0934406B09344
:1024500045068091420690914306A0914406B091B2
:1024600045062091C6013091C7010097A105B1052D
:1024700011F4286001C0277F3093C7012093C60163
:102480000895809139068823A9F48091420690919D
:102490004306A0914406B091450620916B06309109
:1024A0006C0640916D0650916E06820F931FA41F1B
:1024B000B51F16C08130E9F4809142069091430621
:1024C000A0914406B091450620916B0630916C06B0
:1024D00040916D0650916E06821B930BA40BB50BB9
:1024E0008093420690934306A0934406B09345061A
:1024F000D8C0823099F46091420670914306809171
:1025000044069091450620916B0630916C064091EF
:102510006D0650916E060E94B63831C08330D9F4F2
:102520006091420670914306809144069091450661
:1025300020916B0630916C0640916D0650916E06AD
:102540000E94FC3820934206309343064093440691
:1025500050934506A6C08430D9F46091420670912C
:102560004306809144069091450620916B06309178
:102570006C0640916D0650916E060E94FC38609387
:10258000420670934306809344069093450689C0A3
:102590008530A9F48091420690914306A0914406AB
:1025A000B091450620916B0630916C0640916D0606
:1025B00050916E0682239323A423B52391CF8630B6
:1025C000A9F48091420690914306A0914406B091EF
:1025D000450620916B0630916C0640916D06509136
:1025E0006E06822B932BA42BB52B7ACF8730A9F4C0
:1025F0008091420690914306A0914406B091450611
:1026000020916B0630916C0640916D0650916E06DC
:1026100082279327A427B52763CF883069F4809158
:102620006B0690916C06A0916D06B0916E06809538
:102630009095A095B0950AC0893089F480914206A2
:1026400090914306A0914406B091450680936B0695
:1026500090936C06A0936D06B0936E0622C08A30EC
:1026600001F5209142063091430640914406509175
:10267000450680916B0690916C06A0916D06B09115
:102680006E068093420690934306A0934406B0934F
:10269000450620936B0630936C0640936D0650936D
:1026A0006E068091420690914306A0914406B09137
:1026B00045062091C6013091C7010097A105B105DB
:1026C00011F4286001C0277F3093C7012093C60111
:1026D0000895EF92FF920F931F93E0904206F090BF
:1026E000430600914406109145062091BD013091AA
:1026F000BE014091BF015091C0012E153F0540071A
:1027000051073CF48091C6019091C70184608C7F91
:102710000EC08091C6019091C701E216F30604072E
:10272000150719F4897F816002C0887F82609093C9
:10273000C7018093C6018091C6019091C701E11441
:10274000F1040105110511F4886001C0877F9093A1
:10275000C7018093C6011F910F91FF90EF900895DC
:1027600080913906882339F48091C6019091C70180
:1027700083FF7AC060C0813039F48091C6019091A6
:10278000C70183FD71C057C0823029F48091C60112
:102790009091C7012CC0833039F48091C60190918B
:1027A000C70180FD61C047C0843039F48091C60103
:1027B0009091C70182FF58C03EC0853039F48091A6
:1027C000C6019091C70182FD36C011C0863039F430
:1027D0008091C6019091C70181FF46C02CC087300F
:1027E00049F48091C6019091C70181FD24C080FF0A
:1027F0003BC021C0883039F48091C6019091C70157
:1028000084FF32C018C0893039F48091C60190919C
:10281000C70185FF29C00FC08A3039F48091C601F5
:102820009091C70186FF20C006C08B3069F480916B
:10283000C60187FF19C08091BB019091BC019093A4
:1028400037068093360608958C3071F48091C60166
:102850009091C70190FF08C08091BB019091BC018D
:10286000909337068093360608958091BB0190912E
:10287000BC01909337068093360608952091A701F6
:102880002830B8F4E22FF0E0EE0FFF1FE956FE4FBC
:102890008091360690913706918380832F5F209335
:1028A000A7018091BB019091BC0190933706809362
:1028B00036060895E091A701EE2371F0E150E09310
:1028C000A701F0E0EE0FFF1FE956FE4F80819181D6
:1028D00090933706809336060895809139068130AB
:1028E00011F480939601089580913906813011F496
:1028F000109296010895109241060895809139062C
:10290000882339F48091C6019091C7018F7090702F
:102910001FC0813031F48091C6019091C7018F7E34
:1029200017C0823031F48091C6019091C7018F7D2C
:102930000FC0833031F48091C6019091C7018F7B25
:1029400007C0843051F48091C6019091C7018F7700
:102950009093C7018093C6010895853049F4809112
:10296000C6019091C7019E7F9093C7018093C601D5
:10297000089580913906813041F48091CD0580938E
:10298000E3018091CF058093E4010895089500004C
:1029900008950000089500000895000008950000C3
:1029A00008950000089500000895000008950000B3
:1029B00008950000089500000895000008950000A3
:1029C0000895000008950000089500000895000093
:1029D0000895000008950000089500000895000083
:1029E0000895000008950000089500000895000073
:1029F000089510924106089580913906813041F47E
:102A00008091BB019091BC0190933706809336066C
:102A100081E080934106089582E080934106089505
:102A200083E08093410610923706109236068FEFAE
:102A30009FEF9093CB018093CA011092A70110924F
:102A400046061092A80181E08093C3011092C9014B
:102A50001092C8011092420610924306109244064A
:102A60001092450610929601089510924E0610920B
:102A7000C9011092C8010895809139068130D9F0BA
:102A8000813030F0823031F1833009F044C033C0FE
:102A9000809141068093CC05809146068093CB05BA
:102AA0002091C8013091C901832F99278093CD05CA
:102AB0002093CF050895809141068093CC058091A5
:102AC00046068093CB05809137068093CD05809193
:102AD00036060EC0809145068093CC058091440651
:102AE0008093CB05809143068093CD05809142066B
:102AF0008093CF05089580916E068093CC058091D8
:102B00006D068093CB0580916C068093CD058091F6
:102B10006B068093CF0508958091CF058093610166
:102B200081E080931B068091DF05882319F082E005
:102B300080931B0680911606882319F083E080930A
:102B40001B06089586E08093350608958091390626
:102B5000813049F08130A0F0823009F44FC08330D9
:102B600009F063C058C04091E1015091E2016091C9
:102B7000BB017091BC01EDECF1E020E030E03AC027
:102B80002091E1013091E2012A30310590F4F90100
:102B9000EE0FFF1FE353FE4F8091BB019091BC01EC
:102BA000918380832F5F3F4F3093E2012093E101B7
:102BB000089589E080933506089581919191861753
:102BC0009707B1F4F901EE0FFF1FE353FE4F415099
:102BD000504006C02F5F3F4F828193818193919334
:102BE00024173507B8F35093E2014093E1010895AB
:102BF0002F5F3F4F2417350701F708951092E20128
:102C00001092E101EDECF1E01192119281E0E13ED0
:102C1000F80771F0F9CF1092CC051092CB05109205
:102C2000CD058AE08093CF05089583E08093350633
:102C3000089580916406813881F580916506823916
:102C400061F580916606833A41F580916706843B81
:102C500021F580916806853C01F580916906863DE5
:102C6000E1F4F894C098AB9A89E0E3E0F0E0809357
:102C700057008491867019F40C94003808958230BE
:102C800019F40C94003C0895843019F40C94003E1F
:102C90000895863011F40C94003F0895CF93DF938C
:102CA000CDB7DEB728970FB6F894DEBF0FBECDBF05
:102CB000809139068130F1F480913A068A32C1F46C
:102CC0008091CF0589838091CD058A838091CB0542
:102CD0008B838091CC058C831D821E821F82188677
:102CE000BE016F5F7F4F8FEF97E00E9444302FC08F
:102CF00084E02BC0882341F5BE016F5F7F4F8FEFCB
:102D000097E00E940E309091CF058981981799F431
:102D10009091CD058A81981771F49091CB058B81A4
:102D2000981749F49091CC058C81981721F481E093
:102D30008093CF0502C01092CF051092CC0510925F
:102D4000CB051092CD0503C083E08093350628960D
:102D50000FB6F894DEBF0FBECDBFDF91CF910895BF
:102D600080914106882389F1833079F1853069F1BA
:102D700069EA71E080913606909137060E940E3024
:102D800020913606309137068091CA019091CB018F
:102D90008217930721F081E08093C30102C0109253
:102DA000C3013093CB012093CA012F5F3F4F309373
:102DB00037062093360680914106823019F485E06B
:102DC0008093410681E090E0089580E090E00895CE
:102DD0008CE090E00E94790F8093B20180913906D7
:102DE000882399F482E08093C40124E530E0A2EBCB
:102DF000B1E0F9018491FD0181832F5F3F4F11966E
:102E0000F1E0AA3BBF0761F0F4CF1092CC0581E05E
:102E10008093CB0583E08093CD0585E28093CF0539
:102E200008952091BB013091BC013093C9012093DA
:102E3000C80182E08093C4012F5F374078F487E0B7
:102E400090E00E94790F80FD09C063EB71E08091F2
:102E5000C8019091C9010E940E3007C0E2EBF1E079
:102E6000119281E0EB3BF807D9F78CE090E00E94EB
:102E7000790F8093B201089583E08093410687E043
:102E800090E00E94790F81FD04C081E080934E069E
:102E900003C088E0809335068091BB019091BC010E
:102EA0009093C9018093C80108950F931F93CF9306
:102EB000DF93CDB7DEB724970FB6F894DEBF0FBE11
:102EC000CDBFE82FF0E06623C1F189E0689F800163
:102ED00011249F0123703070C901880F991F820F40
:102EE000931F080F191F055E1D4F82E00F3C180746
:102EF00044F081E08093350660E070E080E090E08F
:102F000026C0C80102960E94790F8B83C8010196E2
:102F10000E94790FFE0131968183C8010E94790FCA
:102F200089838B8187FF03C08FEF8C8301C01C8254
:102F300069817A818B819C810AC0EE0FFF1FEE0FA1
:102F4000FF1FE15BF94F608171818281938124963B
:102F50000FB6F894DEBF0FBECDBFDF91CF911F91AA
:102F60000F910895CF93DF93CDB7DEB724970FB6B7
:102F7000F894DEBF0FBECDBF6091390680913A064E
:102F80000E94551769837A838B839C834C8140937D
:102F9000CC053B813093CB052A812093CD059981C7
:102FA0009093CF0580915B068823F9F04093450606
:102FB0003093440620934306909342068091420644
:102FC00090914306A0914406B09145062091C60118
:102FD0003091C7010097A105B10511F4286001C027
:102FE000277F3093C7012093C60124960FB6F8942B
:102FF000DEBF0FBECDBFDF91CF9108958091BB01A1
:103000009091BC01825D944041F460E080E090E0EA
:103010000E94810FF8940C94000008950F931F9361
:10302000CF93DF93CDB7DEB724970FB6F894DEBF0A
:103030000FBECDBF90913906992341F189E0989F49
:103040008001112480913A0623E0829FC00111245F
:10305000080F191F055E1D4F82E00F3C180724F072
:1030600081E08093350632C06091CB05C80102969D
:103070000E94810F6091CD05C80101960E94810FC9
:103080006091CF05C8010E94810F20C08091CB05BF
:103090008B839091CD059A839091CF05998387FF7B
:1030A00003C08FEF8C8301C01C82E0913A06F0E0F0
:1030B000EE0FFF1FEE0FFF1FE15BF94F89819A8131
:1030C000AB81BC8180839183A283B38324960FB6A6
:1030D000F894DEBF0FBECDBFDF91CF911F910F914E
:1030E00008959091390697FF13C08091450680930B
:1030F000CC05809144068093CB0580914306809354
:10310000CD05809142068093CF059F779093390635
:1031100090913906992329F0923019F0933009F0F3
:1031200046C0C39A8BB780648BBFC49A8BB7806448
:103130008BBF992329F48BB78F7B8BBFAF980DC0C2
:10314000923029F48BB78F7B8BBFAE9806C093303B
:1031500021F48BB78F7B8BBFAD9880913A0684307A
:1031600030F08091CC050E9423108093CC05809193
:103170003A06833030F08091CB050E942310809373
:10318000CB0580913A06823030F08091CD050E94C7
:1031900023108093CD058091CF050E94231080934A
:1031A000CF0585B3806E85BB8BB780648BBF809164
:1031B0003906813051F585B3806E85BB8BB780644D
:1031C0008BBFC49A8BB780648BBF8BB78F7B8BBF51
:1031D000C3988091CC050E9423108093CC058091E8
:1031E000CB050E9423108093CB058091CD050E94D2
:1031F00023108093CD058091CF050E9423108093EA
:10320000CF05C39A8BB780648BBF80915B06882300
:1032100059F18091CC05809345068091CB05809330
:1032200044068091CD05809343068091CF0580931D
:1032300042068091420690914306A0914406B091C7
:1032400045062091C6013091C7010097A105B1053F
:1032500031F428603093C7012093C6010895277F79
:103260003093C7012093C60108951F9381E0809396
:10327000460640913906442339F08091BB01909174
:10328000BC011816190604F52091C301222341F050
:103290008091BB019091BC019093C2018093C101C8
:1032A000442391F48091BB019091BC018F5F9F4FAB
:1032B00051F5222341F1809142069091430690936B
:1032C000C2018093C1011FC08091BB019091BC01DC
:1032D000181619061CF020E030E00AC020E08091AA
:1032E000C1019091C201892B09F021E081E02827DA
:1032F000122F8091C6019091C701222311F08061A5
:1033000021C08F7E1FC08091C1019091C201892B85
:1033100011F41092460680914606882341F0809170
:10332000CA019091CB019093370680933606809125
:10333000C6019091C7018F7E9093C7018093C6010B
:1033400010E025C09093C7018093C6014130F9F485
:1033500060E08DE70E94840790E020913A06220FFA
:1033600002C0959587952A95E2F780FF02C01092DA
:10337000460680914606882351F0112341F480913E
:10338000CA019091CB0190933706809336068091C5
:103390003906823019F563E08DE70E94840790E0DA
:1033A00040913A06440F22E030E002C0220F331F62
:1033B0004A95E2F782239323892B11F01092460657
:1033C00080914606882351F0112341F48091CA016F
:1033D0009091CB0190933706809336068091390601
:1033E0008330F9F463E08DE70E94840790E0209138
:1033F0003A06220F02C0959587952A95E2F780FF3D
:1034000002C01092460680914606882351F011238F
:1034100041F48091CA019091CB019093370680933B
:10342000360680913906843009F049C0E0913A06A9
:10343000E33050F410924606F0E0E151FA4F8081FB
:10344000882379F181E028C0E43049F48091EF05C8
:10345000882301F520E030E08091F00515C0E530CB
:1034600059F0E63019F48091EF0508C0E730B9F45F
:103470008091EF05882371F48091F005882351F441
:1034800020E030E08091F105882311F021E030E068
:10349000C90102C081E090E08093460602C010920C
:1034A000460680914606882351F0112341F480910D
:1034B000CA019091CB0190933706809336061F91F5
:1034C000089580913906882341F4E0913A06F0E0AE
:1034D000E151FA4F81E080830895813081F4809139
:1034E0003A06E82FF0E0E151FA4F9FE0908362E066
:1034F0000E947D0880913A060E94CF08089582308C
:1035000049F5E0913A06F0E0E151FA4FE081E093AD
:10351000CF0580915B068823E9F08E2F90E0A0E034
:10352000B0E08093420690934306A0934406B09384
:1035300045068091C6019091C701EE2331F4886061
:103540009093C7018093C6010895877F9093C70128
:103550008093C601089562E080913A060E947D083A
:1035600080913A060E94CF080895EF92FF920F9340
:103570001F93CF93DF9380913A06882341F4809183
:103580003906873109F001C10E943509FEC081303A
:1035900009F0B0C080913906863038F4C82FD0E0E9
:1035A000C759DE4F8330E1F415C0893038F4C82F95
:1035B000D0E0CC0FDD1FCC59DE4F12C08C3008F0AC
:1035C000E1C0C82FD0E0CC0FDD1FCC0FDD1FCC5ADF
:1035D000DE4F06C0CE010E94790F8093CB040FC04E
:1035E000843031F4CE010E94790F8093CA0407C061
:1035F000853029F4CE010E94790F8093CC0480910C
:103600003906863061F4CE0101960E94790F8093CD
:10361000CE04CE010E94790F8093CD04B6C08730CE
:1036200061F4CE0101960E94790F8093C704CE0108
:103630000E94790F8093C604A8C0883061F4CE013F
:1036400001960E94790F8093C904CE010E94790FE0
:103650008093C8049AC08930C1F4CE0103960E94B9
:10366000790F8093B405CE0102960E94790F809362
:10367000B305CE0101960E94790F8093B205CE0169
:103680000E94790F8093B10580C08A30C1F4CE01C9
:1036900003960E94790F8093B805CE0102960E948E
:1036A000790F8093B705CE0101960E94790F809320
:1036B000B605CE010E94790F8093B50566C08B30A8
:1036C00009F063C0CE0103960E94790F8093C50470
:1036D000CE0102960E94790F8093C404CE01019618
:1036E0000E94790F8093C304CE010E94790F8093CA
:1036F000C2044BC0823009F048C00091390608333B
:1037000008F043C010E0000F111F000F111FBBE1B4
:10371000EB2EB3E0FB2EE00EF11EC7010E94790FE5
:1037200000531B4FF801808380913906C82FD0E0E9
:10373000CC0FDD1FCC0FDD1FCF52DB4FC701019631
:103740000E94790F888380913906C82FD0E0CC0F72
:10375000DD1FCC0FDD1FCE52DB4FC70102960E944A
:10376000790F888380913906C82FD0E0CC0FDD1FF8
:10377000CC0FDD1FCD52DB4FC70103960E94790F9E
:10378000888303C0CFEFD3E02BCFDF91CF911F9180
:103790000F91FF90EF9008950F931F93CF93DF93B6
:1037A00080913A06882321F480913906893449F0C2
:1037B00089E090E00E94790F882319F085E08093DA
:1037C000350680913A06882311F5809139068034B8
:1037D00028F5873088F4863011F48EE70AC0880F08
:1037E000880F8C590E946C0A80913906880F880FC7
:1037F0008A590E946C0AF0C0873019F40E942B0A83
:10380000EBC0873109F0E8C00E94EA09E5C08130C9
:1038100009F09FC080913906833020F483E08093C3
:103820003506DAC0863038F4C82FD0E0C759DE4FED
:103830008330C9F415C0893038F4C82FD0E0CC0FDC
:10384000DD1FCC59DE4F0FC08C3008F0C2C0C82F2E
:10385000D0E0CC0FDD1FCC0FDD1FCC5ADE4F03C0F4
:103860006091CB0409C0843019F46091CA0404C08B
:10387000853029F46091CC04CE010E94810F8091A3
:103880003906863049F46091CE04CE0101960E943B
:10389000810F6091CD045BC0873049F46091C7040B
:1038A000CE0101960E94810F6091C60450C08830FD
:1038B00049F46091C904CE0101960E94810F609184
:1038C000C80445C08930A9F46091B405CE010396BF
:1038D0000E94810F6091B305CE0102960E94810F74
:1038E0006091B205CE0101960E94810F6091B105F1
:1038F0002EC08A30A9F46091B805CE0103960E94CB
:10390000810F6091B705CE0102960E94810F6091F0
:10391000B605CE0101960E94810F6091B50517C0D2
:103920008B3009F059C06091C504CE0103960E9406
:10393000810F6091C404CE0102960E94810F6091B4
:10394000C304CE0101960E94810F6091C204CE0192
:103950003DC0823009F040C0E0913906E833E0F51F
:10396000F0E0EE0FFF1FEE0FFF1F8F01055E1C4FF3
:10397000E053FB4F6381C80103960E94810FE091E1
:103980003906F0E0EE0FFF1FEE0FFF1FE053FB4F75
:103990006281C80102960E94810FE0913906F0E031
:1039A000EE0FFF1FEE0FFF1FE053FB4F6181C801B9
:1039B00001960E94810FE0913906F0E0EE0FFF1FA3
:1039C000EE0FFF1FE053FB4F6081C8010E94810F83
:1039D00003C0CFEFD3E047CFDF91CF911F910F917D
:1039E00008950F931F93CF93DF93CDB7DEB728973A
:1039F0000FB6F894DEBF0FBECDBF80913A06882384
:103A000009F0DCC08091390687FD7DC0803408F064
:103A100041C08630A9F48FE78093DB0560EE75E046
:103A20008BED95E00E9457048091E3058093CF05CC
:103A30008091E2058093CD058091E1058093CB05CF
:103A400080913906873008F449C1880F880F8B5957
:103A50008093DB0560EE75E08BED95E00E945704E6
:103A60008091E3058093CF058091E2058093CD0599
:103A70008091DB058E5F8093DB0560EE75E08BED5A
:103A800095E00E9457048091E3058093CB058091D7
:103A9000E20536C0803519F486E090E008C0813533
:103AA00019F487E090E003C090E0805490401092B9
:103AB000CD050E94790F8093CF0590913906892F0B
:103AC0008654823008F00AC1963419F40EE411E0ED
:103AD00002C00AE411E0C8010E94790F8093CF056B
:103AE000C80101960E94790F8093CD05C801029606
:103AF0000E94790F8093CB05C80103960E94790F2D
:103B00008093CC05EBC01092CC051092CB0510929F
:103B1000CD05803819F48091410616C0813819F41A
:103B200080914E0611C0823859F4809136069091EA
:103B30003706892F99278093CD058091360604C0DA
:103B4000833829F48091A8018093CF052FC0843851
:103B5000C9F4F8948091EB059091EC05A091ED05E6
:103B6000B091EE0589839A83AB83BC837894898175
:103B70008093CF058A818093CD058B818093CB057F
:103B80008C8112C0853891F40E94A8386D837E83A1
:103B90008F8398878D818093CF058E818093CD050B
:103BA0008F818093CB0588858093CC0580913906E1
:103BB0008F3F09F093C08091C5018EC0813009F01C
:103BC00074C01092CC051092CB051092CD05809157
:103BD0003906882319F48091CF0415C08130A9F0EB
:103BE000823019F48091B0050EC0833019F48091B1
:103BF000CB0409C0843019F48091CA0404C0853014
:103C000021F48091CC048093CF05809139068630D1
:103C100039F48091CE048093CD058091CD045CC0B1
:103C2000873039F48091C7048093CD058091C60414
:103C300053C0883039F48091C9048093CD058091B8
:103C4000C8044AC0893079F48091B4058093CC05CA
:103C50008091B3058093CB058091B2058093CD050B
:103C60008091B10539C08A3079F48091B80580938C
:103C7000CC058091B7058093CB058091B6058093E4
:103C8000CD058091B50528C08B3041F58091C504E4
:103C90008093CC058091C4048093CB058091C304AC
:103CA0008093CD058091C20417C08230B9F4E091B1
:103CB0003906E83398F4F0E0EE0FFF1FEE0FFF1F18
:103CC000E053FB4F83818093CC0582818093CB05A9
:103CD00081818093CD0580818093CF0580915B06A3
:103CE000882339F18091CC05809345068091CB05DE
:103CF000809344068091CD05809343068091CF0543
:103D0000809342068091420690914306A09144061A
:103D1000B09145062091C6013091C7010097A105D9
:103D2000B10511F4286001C0277F3093C7012093AB
:103D3000C60128960FB6F894DEBF0FBECDBFDF9147
:103D4000CF911F910F910895EF92FF920F931F93C0
:103D5000CF93DF9380913A06882309F01AC18091AE
:103D6000390687FDE4C0803458F5863061F420912F
:103D7000CF05207F6091CB056F7C60624091CD05BF
:103D80008EE70E94510500913906073008F4B1C151
:103D900010E0000F111F000F111F2091CF0540915F
:103DA000CD0560E0802F8C590E9451052091CB05F4
:103DB0004091CC0560E0802F8A590E94510599C13D
:103DC000893409F58091BB019091BC0124E0823DCA
:103DD000920731F41092CD0581E08093CF050CC09D
:103DE000815E904129F41092CD051092CF0504C058
:103DF00084E0809335067DC16091CF0589E090E035
:103E00000E94810F76C1803519F4C6E0D0E015C05C
:103E1000813529F0C82FD0E0C054D0400EC0809129
:103E2000CF0580FD08C087E090E00E94790F80FFF9
:103E300002C00E94922FC7E0D0E0809139068734FB
:103E400019F4CAE4D1E004C0863411F4CEE4D1E020
:103E50008654823090F46091CC05CE0103960E9486
:103E6000810F6091CB05CE0102960E94810F609177
:103E7000CD05CE0101960E94810F6091CF05CE0144
:103E80000E94810F80913906873411F0853449F5FD
:103E90008AE491E00E94790F80932F068BE491E0F1
:103EA0000E94790F809330068CE491E00E94790F94
:103EB000809331068DE491E00E94790F8093320661
:103EC000E0902F06F09030060091310610913206F6
:103ED00085E090E00E94790FB801A70190E00E9470
:103EE000DD33809139068634C1F48EE491E00E947E
:103EF000790F8093E7058FE491E00E94790F80931A
:103F0000E80580E591E00E94790F8093E90581E55D
:103F100091E00E94790F8093EA05809139068234FE
:103F200009F0E7C08091CF050E947236E2C0833865
:103F300029F48091CF058093A80121C0843899F499
:103F4000F8948091BD019091BE01A091BF01B09104
:103F5000C0018093EB059093EC05A093ED05B09321
:103F6000EE0578940CC0853851F46091BD017091D4
:103F7000BE018091BF019091C0010E94AD38809137
:103F800039068F3F09F0B5C08091CF058093C501F8
:103F9000B0C0813009F094C080913906882329F49B
:103FA0008091CF058093CF04A4C0813009F44FC025
:103FB000823029F48091CF058093B0059AC0833078
:103FC00029F48091CF058093CB0493C0843029F4E9
:103FD0008091CF058093CA048CC0853029F48091EC
:103FE000CF058093CC0485C0863079F48091CD05CF
:103FF00090E0982F88272091CF0530E0822B932BDB
:104000009093CE048093CD0474C0873079F480916E
:10401000CD0590E0982F88272091CF0530E0822BA6
:10402000932B9093C7048093C60463C0883079F4BF
:104030008091CD0590E0982F88272091CF0530E022
:10404000822B932B9093C9048093C80452C089306B
:1040500089F48091BD019091BE01A091BF01B09102
:10406000C0018093B1059093B205A093B305B093BE
:10407000B4053FC08A3089F48091BD019091BE01A2
:10408000A091BF01B091C0018093B5059093B60592
:10409000A093B705B093B8052CC08B3051F5809133
:1040A000BD019091BE01A091BF01B091C00180936C
:1040B000C2049093C304A093C404B093C50419C070
:1040C0008230B9F4E0913906E83398F4F0E0EE0F6D
:1040D000FF1FEE0FFF1FE053FB4F8091CC05838342
:1040E0008091CB0582838091CD0581838091CF051E
:1040F0008083DF91CF911F910F91FF90EF900895F2
:10410000309145063093CC05209144062093CB0591
:10411000909143069093CD05809142068093CF0500
:104120009093BC018093BB013093C0012093BF01E9
:104130009093BE018093BD010E94A41E08950F9329
:104140001F93CF93DF93E0913906E7FD08C0EF306E
:1041500008F0B9C0F0E0E059FE4FE49101C0EF77FC
:10416000E0933906909139069034C8F4E92FF0E0D5
:1041700000913A069F3040F4EE0FFF1F0295000FAA
:10418000007E802F8E2B08C0EB5AFE4F8491880F43
:104190000295000F007E802B0E94B60A94C09B34CB
:1041A000E1F480913A06C82FD0E0CC0FDD1FCE019C
:1041B000865A9E4F0E94790FC05FD94F88838091A5
:1041C0003A06C82FD0E0CC0FDD1FCE01855A9E4F96
:1041D0000E94790FC05FD94F1DC09C34E9F48091D3
:1041E0003A06C82FD0E0CC0FDD1FCE01805A9E4F7B
:1041F0000E94790FCE50DA4F888380913A06C82FFB
:10420000D0E0CC0FDD1FCE018F599E4F0E94790F59
:10421000CE50DA4F898357C09335E1F480913A0646
:10422000C82FD0E0CC0FDD1FCE018A599E4F0E94CF
:10423000790FC55ADE4F888380913A06C82FD0E0A7
:10424000CC0FDD1FCE0189599E4F0E94790FC55AB0
:10425000DE4FE0CF892F8155823020F483E08093B8
:10426000350631C000913A069D3459F410E0C8017A
:1042700083509C4F0E94790F095E194FF80180838B
:1042800022C0C02FD0E0C05CD04083E0989FC00126
:104290001124C80FD91FCE0140960E94790F809338
:1042A000CF05682F8C2F0E94071080913906853426
:1042B00051F4CE010D960E94790F682F9E01235074
:1042C000822F0E940710DF91CF911F910F910895C7
:1042D0001F93CF93DF93E0913906E7FD08C0EF30DD
:1042E00008F0B3C0F0E0E059FE4FE49101C0EF7771
:1042F000E0933906209139062034D0F4E22FF0E023
:1043000090913A062F3040F4EE0FFF1F9295990FCF
:10431000907E892F8E2B08C0EB5AFE4F8491880F18
:104320009295990F907E892B0E946C0A182F88C055
:104330002B34C9F480913A0690E0880F991FFC0154
:10434000E05FF94F6081865A9E4F0E94810F8091F5
:104350003A0690E0880F991FFC01E05FF94F6181F8
:10436000855A9E4F1AC02C34D9F480913A0690E0B9
:10437000880F991FFC01EE50FA4F6081805A9E4FC2
:104380000E94810F80913A0690E0880F991FFC01EE
:10439000EE50FA4F61818F599E4F0E94810F55C098
:1043A0002335C9F480913A0690E0880F991FFC01EB
:1043B000E55AFE4F60818A599E4F0E94810F80917D
:1043C0003A0690E0880F991FFC01E55AFE4F618183
:1043D00089599E4FE2CF2D3451F480913A0690E0F6
:1043E000FC01E95EF94F608183509C4FD6CF822F4C
:1043F0008155823010F483E026C080913A06C82FA0
:10440000D0E0C05CD04083E0289FC0011124C80FD9
:10441000D91F8C2F0E940010682FCE0140960E9459
:10442000810F182F80913906853451F49E01235055
:10443000822F0E940010682FCE010D960E94810FDE
:10444000123019F485E080933506DF91CF911F91EA
:104450000895DF92EF92FF920F931F93CF93DF9314
:10446000CDB7DEB726970FB6F894DEBF0FBECDBF2F
:10447000E0913906E7FD08C0EF3008F00FC2F0E028
:10448000E059FE4FE49101C0EF77E09339062091A7
:1044900039062B3108F0B3C0233041F4E0913A06DD
:1044A000F0E0EE0FFF1FE35AF94F09C0263061F428
:1044B000E0913A06F0E0EE0FFF1FE95BF94F8181D2
:1044C0008093CD05808190C090913A06E22FF0E074
:1044D000293058F5EE0FFF1F9295990F907E9E2B75
:1044E00091609093DB0560EE75E08BED95E00E94A6
:1044F00057048091E1058093CB059091E20590935C
:10450000CD058091E3058093CF05809139068430F5
:1045100008F46CC093FF6AC0906F9093CD058FEF45
:104520008093CB058093CC0561C0EB5AFE4F8491FC
:10453000880F9295990F907E982B91609093DB0550
:1045400060EE75E08BED95E00E9457041E8280912D
:10455000E1058D838091E2058C838091E3058B8357
:104560002B813C814D815E81E09139068E2F90E058
:10457000FC01ED5BFE4FE49104C0559547953795DE
:104580002795EA95D2F72B833C834D835E83815D2B
:104590009E4FEE24FF24870160E070E0FC01D49080
:1045A0000FC081E090E0A0E0B0E004C0880F991F48
:1045B000AA1FBB1FEA95D2F7E82AF92A0A2B1B2B60
:1045C000E62F6F5F7F4FED1560F3E222F3220423A5
:1045D0001523EB82FC820D831E838D818093CB0596
:1045E0008C818093CD058B818093CF058091CB0505
:1045F00087FF02C08FEF25C11092CC0524C12E3158
:1046000008F03FC01092CC051092CB051092CD055A
:104610001092CF058DE78093DB0560EE75E08BEDA2
:1046200095E00E945704809139068B3199F480916E
:104630003A06880F22E030E002C0220F331F8A952D
:10464000E2F78091E30590E028233923232B09F436
:10465000FAC015C08C3119F48091E30505C08D3185
:1046600009F0F1C08091E00590E020913A06220F18
:1046700002C0959587952A95E2F780FFE4C081E016
:10468000A0C0203408F4DFC0203608F09DC010918F
:104690003A06105C83E0289FC0011124180F2534CE
:1046A00031F4812F83500E9400108093CD05812F1B
:1046B0000E9400108093CF05809139068B34A9F4B5
:1046C000E0913A06F0E0EE0FFF1FE05FF94F9181B5
:1046D0009093CD0580818093CF0597FF27C08FEF02
:1046E0008093CC058093CB0521C08C3441F4E091BC
:1046F0003A06F0E0EE0FFF1FEE50FA4F09C0833587
:1047000059F4E0913A06F0E0EE0FFF1FE55AFE4F34
:1047100081818093CD0507C0863541F4E0913A064A
:10472000F0E0E05AFF4F80818093CF0580913906F9
:104730008D3431F4E0913A06F0E0E95EF94F0FC0B4
:104740008E3431F4E0913A06F0E0EC51FA4F07C0B4
:10475000803541F4E0913A06F0E0E350FA4F808171
:104760008093CF05809139068135A1F480913A0676
:104770000E9414386B837C838D839E838E8180930B
:10478000CC058D818093CB058C818093CD058B8169
:104790008093CF0580913906873419F0803409F071
:1047A00052C09091CF0584E6989FC001112461E129
:1047B00070E00E94D5387A8369838A818093CD0521
:1047C00089818093CF053FC02236C1F41092CD0578
:1047D000E0913A06F0E0E25CF94F808181FF04C08D
:1047E00081E08093CF0502C01092CF05E0913A0698
:1047F000F0E0E25CF94F80818D7F80838091390603
:104800008336C1F41092CD05E0913A06F0E0E25C07
:10481000F94F808182FF04C081E08093CF0502C000
:104820001092CF05E0913A06F0E0E25CF94F80810A
:104830008B7F80838091CD0587FF05C08FEF8093AC
:10484000CB058093CC0580915B06882339F180915C
:10485000CC05809345068091CB05809344068091DA
:10486000CD05809343068091CF05809342068091C9
:10487000420690914306A0914406B09145062091CE
:10488000C6013091C7010097A105B10511F4286058
:1048900001C0277F3093C7012093C60126960FB62B
:1048A000F894DEBF0FBECDBFDF91CF911F910F9166
:1048B000FF90EF90DF9008950F931F93CF93DF93B6
:1048C000982FC82FDD27C7FDD095FE01E55CF94F75
:1048D0008081882319F480E090E01EC010828E0150
:1048E000000F111FF801E95BF94F60817181892F79
:1048F0000E94F107035A194F25E0CC0FDD1F2A95BE
:10490000E1F7F8012081418160E0FE01E6608E2F31
:104910000E94510581E090E0DF91CF911F910F91AE
:104920000895CF93DF93CDB7DEB722970FB6F894F3
:10493000DEBF0FBECDBF90913A06E92FF0E0E55CF7
:10494000F94F8081813019F4892F0E945C24809175
:10495000BB019091BC01909581959F4F9A8389836B
:1049600062E080913A060E947D0880913A06829525
:10497000880F807E29814A8160E088600E9451050D
:1049800080913A068295880F807E2FEF47E060E0A5
:1049900086600E945105E0913A06F0E0E55CF94F2F
:1049A00082E0808322960FB6F894DEBF0FBECDBFA3
:1049B000DF91CF91089590913A06E92FF0E0E55C00
:1049C000F94F8081813019F4892F0E945C2462E0C4
:1049D00080913A060E947D0880913A068295880F60
:1049E000807E2091CF054091CD0560E088600E94D7
:1049F000510580913A068295880F807E2FEF47E01F
:104A000060E086600E945105E0913A06F0E0E55CC6
:104A1000F94F82E080830895DF92EF92FF920F9327
:104A20001F93CF93DF93CDB7DEB724970FB6F894DB
:104A3000DEBF0FBECDBFD62E082F10E0C801E5E0C7
:104A4000880F991FEA95E1F782600E94C2079B01D7
:104A5000AC01DD2069F17801EE0CFF1CE00EF11EC7
:104A60008BE192E0E80EF91E89E0D89EC001112486
:104A7000E80EF91E9FECE91692E0F90624F081E0B9
:104A80008093350620C029833A834B835C836B81F6
:104A9000C70102960E94810FFE0131966181C70114
:104AA00001960E94810F6981C7010E94810F0BC08E
:104AB000000F111F000F111F015B194FF801208318
:104AC00031834283538324960FB6F894DEBF0FBE22
:104AD000CDBFDF91CF911F910F91FF90EF90DF90AD
:104AE00008951F931091390680913A06833010F48F
:104AF000612F30C0843041F4612F80E00E940C258A
:104B0000612F81E00E940C2580913A06853041F4A6
:104B1000612F81E00E940C25612F82E00E940C250C
:104B200080913A06863041F4612F80E00E940C2586
:104B3000612F82E00E940C2580913A06873061F453
:104B4000612F80E00E940C25612F81E00E940C25DE
:104B5000612F82E00E940C251F910895CF92DF9271
:104B6000EF92FF920F931F93182F062F8295880FB5
:104B7000807E82600E94C2076B017C01602F812FC2
:104B80000E9455176C157D058E059F0529F460E080
:104B900070E080E090E010C0C616D706E806F9067F
:104BA0002CF46C197D098E099F0906C0C61AD70A14
:104BB000E80AF90AC701B6011F910F91FF90EF9023
:104BC000DF90CF9008950F931F93182F062F60E06A
:104BD0000E947D08602F812F0E945517AB01BC01F8
:104BE000812F8295880F807E0E9499081F910F91D6
:104BF00008954F925F926F927F928F929F92AF92A1
:104C0000BF92CF92DF92EF92FF920F931F93CF93B9
:104C1000DF93CDB7DEB728970FB6F894DEBF0FBE8F
:104C2000CDBF4091CC0548872091CB052F83309193
:104C3000CD053E838091CF058D83E0913906E7FD58
:104C400008C0EF3008F09EC1F0E0E059FE4FE4915B
:104C500001C0EF77E0933906E0913906E73411F0AF
:104C6000E03479F48091BB019091BC0153E0880F4E
:104C7000991F5A95E1F76FE270E00E94E93860935E
:104C8000CF05E03408F0E8C0E930B0F5E63081F453
:104C90006091BB017091BC0180913A060E94F107BE
:104CA000E0913A06F0E0EE0FFF1FE95BF94FDDC03F
:104CB0002093DC053093DD058091CF058093DE05E0
:104CC000EE0F80913A068295880F807E8E2B80931E
:104CD000DB0560EE75E08BED95E00E945704809156
:104CE0003906833009F042C1E0913A06F0E0EE0F58
:104CF000FF1FE35AF94FB9C0E031E9F480913A0659
:104D00008295880F807E81618093DB0560EE75E07F
:104D10008BED95E00E94570480913A068295880FAA
:104D2000807E80618093DB059091CF059F7080919C
:104D3000E105807F1FC090913A06E13169F59295B7
:104D4000990F907E91619093DB0560EE75E08BED9D
:104D500095E00E94570480913A068295880F807EE4
:104D600080618093DB059091CF059295907F809133
:104D7000E1058F70982B9093DC058091E20580937C
:104D8000DD058091E3058093DE0560EE75E08BED37
:104D900095E00E945704EAC01C822B833A838091DD
:104DA000CF058983F0E0EB5AFE4FE491EE0FB92E68
:104DB000B294BB0C90EEB922BE2A8B2D0E94C20782
:104DC000AB01BC01E09139068E2F90E0FC01ED5B58
:104DD000FE4FE49101E010E020E030E004C0000F5D
:104DE000111F221F331FEA95D2F7C980DA80EB80AA
:104DF000FC8044245524815D9E4FFC01A49025C075
:104E00003601470104C095948794779467948A95F6
:104E1000D2F7D401C30181709070892B29F0402B07
:104E2000512B622B732B0AC0D901C8018095909534
:104E3000A095B095482359236A237B23000F111FA7
:104E4000221F331F0894411C511C842D4A14C0F2A8
:104E50008B2D0E9499088AC0EB3471F4E0913A06D8
:104E6000F0E0EE0FFF1FE05FF94F8091BB019091E2
:104E7000BC01918380837AC0EC3441F4E0913A061E
:104E8000F0E0EE0FFF1FEE50FA4FEFCFE33541F4A5
:104E9000E0913A06F0E0EE0FFF1FE55AFE4FE5CF36
:104EA000E63531F4E0913A06F0E0E05AFF4F07C0F2
:104EB000ED3449F4E0913A06F0E0E95EF94F809173
:104EC000CF05808353C0E13579F44C832B833A833B
:104ED0008091CF05898349815A816B817C81809142
:104EE0003A060E94513742C0E235C1F44C832B830D
:104EF0003A838091CF05898369817A818B819C81F6
:104F0000462F4F71F5E09595879577956795FA95BA
:104F1000D1F780913A060E94773728C0E03630F505
:104F200010913A06105C83E0E89FC0011124180F2D
:104F3000E53429F4632F812F83500E94071060917C
:104F4000CF05812F0E94071080913A068B5E0E9448
:104F50000010682F80913A060E94480F8091390610
:104F6000873411F0803411F41092CD058885809338
:104F7000CC058F818093CB058E818093CD058D816B
:104F80008093CF0528960FB6F894DEBF0FBECDBF35
:104F9000DF91CF911F910F91FF90EF90DF90CF9015
:104FA000BF90AF909F908F907F906F905F904F9049
:104FB0000895309145063093CC0520914406209306
:104FC000CB05909143069093CD0580914206809346
:104FD000CF059093BC018093BB013093C001209317
:104FE000BF019093BE018093BD010E94F9250895F1
:104FF0001092CC051092CB051092CD0580913A0607
:10500000882331F580913906883018F40E94130FF7
:105010001DC08A30A0F40E94450F90E0209139060F
:1050200030E02850304002C0959587952A95E2F7E8
:1050300080FF02C081E00AC01092CF0509C083B38F
:1050400090E0969587959695879581708093CF058A
:1050500080913A06813081F4E0913906F0E0EE0F5C
:10506000FF1FE050FA4F208131818181837080934E
:10507000CD052093CF0508C0823031F480913906E8
:105080000E94370F8093CF0580915B06882359F1EA
:105090008091CC05809345068091CB058093440692
:1050A0008091CD05809343068091CF058093420681
:1050B0008091420690914306A0914406B091450626
:1050C0002091C6013091C7010097A105B10531F4C7
:1050D00028603093C7012093C6010895277F30933D
:1050E000C7012093C601089580913A06882339F4B8
:1050F0006091CF05809139060E941D0F089582307E
:1051000071F48091CF0580FF05C0809139060E941F
:105110000B0F0895809139060E940F0F08958F3F5D
:1051200021F56091CF0580E00E94B8046091CD0523
:1051300081E00E94B8046091CB0582E00E94B8042F
:105140008091CF0582FF03C080E00E94CF0880914C
:10515000CD0582FF03C081E00E94CF088091CB057E
:1051600082FF03C082E00E94CF0808950F931F932F
:10517000CF93DF93CDB7DEB72F970FB6F894DEBF8E
:105180000FBECDBF8091B90590913E06892B8093CB
:105190003E0680913F069091BA05892B80933F0689
:1051A0008091BB0590914006892B809340068091A9
:1051B0001A06882349F08091C6019091C701916039
:1051C0009093C7018093C6018091330680FF0BC086
:1051D0008091C1019091C201009729F001979093AD
:1051E000C2018093C1010E947609282F8093EF01AC
:1051F0004091ED015091EE014130510519F08823A5
:1052000009F483C03091DF05832F8150823010F084
:105210002230E1F58091E7059091E805A091E9053C
:10522000B091EA058C839D83AE83BF831A821B8273
:105230002230C1F0313011F497E001C098E0E3EB87
:10524000F1E0DE01189681918D9321E0EB3BF207AE
:10525000D1F79983CE0101960E94A434882309F4E2
:1052600050C222C0EEE1F6E0DE01189681918D93E6
:1052700086E0E632F807D1F787E08983CE01019610
:105280000E94A434882309F43CC23CC080911606D5
:10529000882319F4233091F40DC0233059F068E0CD
:1052A00083EB91E00E949C368091ED019091EE019C
:1052B0008E7F23C268E08EE196E0F4CF8091F805FE
:1052C000882309F01EC2213091F04E7F5093EE01E9
:1052D0004093ED0102EB11E0F80181918F010E94F2
:1052E000372FF1E00B3B1F0709F40BC2F5CF0DE19F
:1052F00016E0F80181918F010E94372FF6E0063207
:105300001F07B9F71092EF01FCC11092CC0183E6A0
:1053100096E00E949D06813069F58093CC018091D2
:10532000630680936F0680916406809339068091AE
:10533000650680933A06809166068093CC0580913D
:1053400067068093CB05809168068093CD05809198
:1053500069068093CF0580914106882319F481E086
:1053600090E053C020E030E0833011F421E030E0E1
:10537000C9014BC08091330682FF23C08091410652
:10538000813009F044C090919601913009F03FC0FE
:1053900083E08093CC0187E180936F0610923906F9
:1053A00010923A061092CC051092CB058091E30141
:1053B0008093CD058091E4018093CF0590935B06A7
:1053C00026C00E94B016882311F182E08093CC01A0
:1053D0008091A90180936F068091AA01809339067C
:1053E0008091AB0180933A068091AC018093CC050B
:1053F0008091AD018093CB058091AE018093CD0566
:105400008091AF018093CF0581E080935B0680910E
:10541000CC01882309F475C182E090E00E94790FE5
:10542000382F80934D062091CD052093BC0190919B
:10543000CF059093BB018091CC058093C0018091F2
:10544000CB058093BF012093BE019093BD011092C4
:10545000350690916F06892F8854883310F09E3856
:1054600070F08091CC01813011F4923F41F082E0E4
:10547000809335068091A80181608093A801809176
:10548000CC01813091F4E3E6F6E08191380F26E01B
:10549000EA36F207D1F730934D0680916A06381745
:1054A000C9F081E08093350615C0823099F4E9EAAD
:1054B000F1E08191380F81E0E03BF807D1F73093BC
:1054C0004D068091B001381729F08091A8018260C3
:1054D0008093A8011092C40180913506882309F0B9
:1054E00095C080914E06882311F097FF50C0923FDF
:1054F00021F40E94191682E087C0E92FF0E097FF9F
:1055000005C0EE0FFF1FED50F04004C0EE0FFF1F6F
:10551000ED59FF4F0190F081E02D84E68093350630
:105520008091F001882311F0099503C08FEF8093DB
:1055300035066091E1017091E2016115710509F490
:1055400065C080914106813009F060C08091CC0136
:10555000823009F05BC0409136065091370620E05A
:1055600030E00FC02F5F3F4FEE0FFF1FE353FE4FA2
:10557000808191814817590721F485E08093410685
:1055800045C0E22FF0E0E617F70760F33FC08091D7
:10559000C8019091C901E7E08F3F9E07A0F563E63F
:1055A00076E00E944430882371F565EE71E08091C9
:1055B000C8019091C9010E940E3085E6809335069E
:1055C00020E030E0F901EB51FE4FD901AD59B94F60
:1055D00090818C91981721F087E08093350605C063
:1055E0002F5F3F4F2830310569F7809135068536AA
:1055F00069F48091C8019091C90101969093C90105
:105600008093C80103C087E0809335068091CC0168
:10561000813009F076C08CE090E00E94790F182F5D
:1056200082E090E00E94790F282F809338068091C5
:10563000C4018823C9F590916F06963031F48091AA
:10564000CB05880F880B8093CC051093B201209373
:10565000B301809135068093B4019093B501809198
:10566000CC058093B6018091CB058093B7018091E2
:10567000CD058093B8018091CF058093B9018091C9
:105680001606882339F010924D0690914D06E3EBF3
:10569000F1E003C010934D06F8CF8191980F21E0FF
:1056A000EA3BF207D1F70FC0813089F41093B201C1
:1056B00010924D06E2EBF1E090E08191980F81E0CD
:1056C000EA3BF807D1F790934D069093BA018BE02F
:1056D00090E00E94790F8093F8058091C50188239E
:1056E00051F080916F06863031F08A3021F08F3092
:1056F00011F08F3131F481E090E09093EE018093CE
:10570000ED012F960FB6F894DEBF0FBECDBFDF912F
:10571000CF911F910F9108959F92AF92BF92CF9218
:10572000DF92EF92FF920F931F93CF93DF93CDB74A
:10573000DEB722970FB6F894DEBF0FBECDBF6C0167
:105740007B01042F6115710509F499C0009709F4D4
:1057500096C06817790709F492C0142F1295110F9B
:10576000107EA6E09A2E912A892D0E94A8079A837E
:105770008983812F8C600E94A8075C0180E0D7FCA0
:1057800007C0EE0CFF1CCC0CDD1C8F5F8F30B9F70F
:10579000E114F10419F471E0E72EF12C40E050E03F
:1057A00001C07901142F4F5F5F4FC70180709E7F4A
:1057B000970136952795892BA1F7C9018C0D9D1D61
:1057C000B7010E94D538FB01672B11F4E1E0F0E04E
:1057D00089819A8154E0880F991F5A95E1F7BF019A
:1057E0000E94D5389B01C50144E0880F991F4A9556
:1057F000E1F7BF010E94D538412F50E0153090F4F9
:1058000084E090E0841B950B082E02C03695279506
:105810000A94E2F73A83298302C0769567958A95C0
:10582000E2F70FC0CA010497082E02C0220F331FEF
:105830000A94E2F73A83298302C0660F771F8A959C
:10584000E2F789819A81892B21F481E090E09A83A3
:1058500089836115710511F461E070E0749718F4A3
:10586000802F0E94F10729814A8160E0892D0E94E2
:105870005105E02FF0E0E55CF94F81E0808322964E
:105880000FB6F894DEBF0FBECDBFDF91CF911F9151
:105890000F91FF90EF90DF90CF90BF90AF909F90CF
:1058A00008950F931F93CF93DF93CDB7DEB7629721
:1058B0000FB6F894DEBF0FBECDBF082F162F843071
:1058C000C1F480E00E945C2481E00E945C24612F8E
:1058D00080E00E94AE256F83788789879A87612F41
:1058E00081E00E94AE256B877C878D879E87198A11
:1058F0003FC0853041F481E00E945C2482E00E9438
:105900005C24198625C0863081F480E00E945C24E6
:1059100082E00E945C24612F80E00E94AE256F83AC
:10592000788789879A871D861BC0873009F580E0B4
:105930000E945C2481E00E945C2482E00E945C243E
:10594000612F80E00E94AE256F83788789879A87D0
:10595000612F81E00E94AE256B877C878D879E87B3
:10596000612F82E00E94AE256F87788B898B9A8B9E
:105970009985992331F48D85882319F489898823A1
:1059800069F09A83FE013796818189838D858C83A6
:105990008C858B8389898E8388890BC088858A83CF
:1059A0008F8189838C858C838B858B8388898E837B
:1059B0008F858D83043049F429813A818B819C81C4
:1059C00082179307D0F441E015C0053049F42B81CC
:1059D0003C818D819E818217930758F041E00EC073
:1059E000063071F429813A818D819E818217930757
:1059F00020F442E0BC01C90133C040E0B90130C02D
:105A0000073081F589819A812B813C81ED81FE816E
:105A10002817390768F4E817F907C0F441E0B9011D
:105A20000E948C2B6D817E8142E089819A8118C011
:105A3000E217F30758F440E0BC01C9010E948C2B27
:105A40006D817E8142E08B819C810AC040E0BC0177
:105A5000CF010E948C2B6B817C8141E08D819E81E6
:105A60000E948C2B62960FB6F894DEBF0FBECDBF9E
:105A7000DF91CF911F910F910895CF92DF92EF9216
:105A8000FF920F931F93CF93DF93CDB7DEB7249789
:105A90000FB6F894DEBF0FBECDBF809139068230BD
:105AA00008F04BC060E080913A060E947D0880912A
:105AB0003A060E945C246E010894C11CD11C80919E
:105AC000CC058C838091CB058B838091CD05F6012D
:105AD00081838091CF05898380913906813009F5D2
:105AE000E980FA800B811C8180913A068295880FAB
:105AF000807E82600E94C207E60EF71E081F191FF3
:105B0000E982FA820B831C838C818093CC058B8184
:105B10008093CB05F60181818093CD0589818093A7
:105B2000CF0549815A816B817C8180913A068295AB
:105B3000880F807E0E94990846C0823009F043C0D9
:105B4000E090CF0580913A06833030F40E945C24C7
:105B50006E2D80913A0635C06E2D0E94512C809199
:105B60003A06843041F46E2D80E00E94E3256E2DCC
:105B700081E00E94E32580913A06853041F46E2D44
:105B800081E00E94E3256E2D82E00E94E325809152
:105B90003A06863041F46E2D80E00E94E3256E2D9A
:105BA00082E00E94E32580913A06873061F46E2DF1
:105BB00080E00E94E3256E2D81E00E94E3256E2D9A
:105BC00082E00E94E32524960FB6F894DEBF0FBE54
:105BD000CDBFDF91CF911F910F91FF90EF90DF909C
:105BE000CF900895CF92DF92EF92FF920F931F9381
:105BF000CF93DF9310923706109236068FEF9FEF08
:105C00009093CB018093CA018DE090E00E94790FC0
:105C1000813011F48093410617E4C12E16E0D12E95
:105C2000BDE5EB2EB6E0FB2EC0E0D0E0CE018295C4
:105C3000880F807E182F8C600E94A807F601819340
:105C400091936F01812F86600E94A807F7018193CD
:105C500091937F012196C330D10541F700ED14E007
:105C6000CEE1D3E0CE010E94790FF8018383CE010B
:105C700001970E94790FF8018283CE0102970E945A
:105C8000790FF8018183CE0103970E94790FF80103
:105C9000808324960C5F1F4FF3E0CE3FDF0711F7A0
:105CA000ECEFFFE7E491E73299F4EDEFFFE7E491E1
:105CB000E83171F4EEEFFFE7E491E83249F4EFEFF9
:105CC000FFE7E491E83121F481E08093F00102C024
:105CD0001092F001DF91CF911F910F91FF90EF9003
:105CE000DF90CF9008951F920F920FB60F9211245C
:105CF0008F939F93EF93FF938BB1887129F08091DD
:105D0000F10180628093F101869B04C08CB1809385
:105D100023021AC080910D029CB1E82FF0E0EE50F2
:105D2000FE4F90838F5F80930D028B3110F01092A5
:105D30000D0290910D0280910E02981729F4809126
:105D4000F10180688093F101FF91EF919F918F9114
:105D50000F900FBE0F901F9018951F920F920FB6C5
:105D60000F9211248F939F93EF93FF9390912202B0
:105D700080912102981781F0969AE92FF0E0E15F77
:105D8000FD4F80818CB9892F8F5F809322028231F1
:105D900020F01092220201C05598FF91EF919F913F
:105DA0008F910F900FBE0F901F9018951F920F921A
:105DB0000FB60F9211248F939F939091220280919E
:105DC0002102981709F496989F918F910F900FBE1A
:105DD0000F901F901895982F80910D0280930E02BE
:105DE00080912202809321021092F1012091D4052A
:105DF000283019F4EEE7F1E002C0E7E8F1E0849121
:105E000089B988ED8AB9992369F0993058F4E92F56
:105E1000F0E0283019F4E258FE4F02C0E957FE4F77
:105E2000849189B908958091F10181FF02C0109297
:105E3000F1018BB1887129F08091F101806280932A
:105E4000F1018091F10182608093F101807F19F06E
:105E50008FEF9FEF089520E030E090910E02809147
:105E60000D02981711F021E030E0C9010895969ACB
:105E700090912102E92FF0E0E15FFD4F80839F5F69
:105E800090932102923110F0109221029091210200
:105E900080912202981729F48091F1018064809307
:105EA000F101559A0895DC0190910E0280910D0246
:105EB000981719F480E090E00895E92FF0E0EE5093
:105EC000FE4F80818C93892F8F5F80930E028B31E0
:105ED00018F481E090E0089510920E0281E090E0C5
:105EE0000895209121022E5F30912202223138F054
:105EF00080E090E0332349F481E090E0089580E071
:105F000090E0231711F481E090E0089520E030E064
:105F10009091220280912102981711F421E030E043
:105F2000C9010895EF92FF920F931F93CF93DF93D0
:105F3000CDB7DEB722970FB6F894DEBF0FBECDBF48
:105F40001A8219827E010894E11CF11C46C08BB7AD
:105F50008F7B8BBFC49886E00E942310C49A8BB7B6
:105F600080648BBF8BB78F7B8BBFC49882E00E940D
:105F70002310F70181810E94231089810E94231040
:105F800000E010E089819A81800F911F885F9F4314
:105F900040F480E00E9423100F5F1F4F0034110572
:105FA00089F7C49A8BB780648BBF00E010E01CC0F7
:105FB000C49A8BB780648BBF0AC0C49A8BB78064C5
:105FC0008BBF0F5F1F4F2EE2003E120769F48981DD
:105FD0009A81805C9F4F9A83898389819A818050BE
:105FE000904408F4B4CF0DC08BB78F7B8BBFC4989F
:105FF00085E00E94231080E00E94231080FDDDCF09
:10600000D7CF22960FB6F894DEBF0FBECDBFDF917B
:10601000CF911F910F91FF90EF900895EF92FF9213
:106020000F931F93CF93DF937B018C0193E0000FBD
:10603000111F9A95E1F78BB78F7B8BBFC49883E0D4
:106040000E942310812F99270E942310802F0E94E5
:106050002310C0E0D0E087010C0F1D1F80E00E94DC
:106060002310F80180832196C830D105A1F7C49A86
:106070008BB780648BBF80E090E0DF91CF911F9160
:106080000F91FF90EF900895EF92FF920F931F935F
:10609000CF93DF937B018C0133E0000F111F3A9502
:1060A000E1F78BB78F7B8BBFC49886E00E942310EB
:1060B000C49A8BB780648BBF8BB78F7B8BBFC49820
:1060C00082E00E942310812F99270E942310802FA5
:1060D0000E942310C0E0D0E0F701EC0FFD1F80818B
:1060E0000E9423102196C830D105B1F7C49A8BB70E
:1060F00080648BBFC0E0D0E013C0C49A8BB78064CB
:106100008BBF80E090E019C0C49A8BB780648BBFCE
:1061100021968EE2C03ED80719F48FEF9FEF0DC095
:106120008BB78F7B8BBFC49885E00E94231080E0E3
:106130000E94231080FDE8CFE0CFDF91CF911F9127
:106140000F91FF90EF9008959091E30596959093AD
:10615000E3058091E20580FF03C090689093E3051A
:106160009091E20596959093E2058091E10580FF7C
:1061700003C090689093E2058091E1058695809335
:10618000E10586FF03C080688093E1050895E82F4C
:10619000F0E0EE0FFF1FEB5CFD4F808191810097D7
:1061A00019F00197918380830895BF92CF92DF9277
:1061B000EF92FF920F931F93CF93DF93082FC82E78
:1061C000DD24F601E151FA4F108123E0B22EB80E22
:1061D0008B2D0E940010E601CC0FDD1F843098F457
:1061E0008DE70E949B0722E030E00C2E02C0220FB8
:1061F000331F0A94E2F7F82EF2228DE70E949B07E4
:1062000021E030E012C08DE70E949B0721E030E0E2
:106210000C2E02C0220F331F0A94E2F7F82EF2224E
:106220008DE70E949B0722E030E002C0220F331F5F
:10623000CA95E2F78223E02EE294EE0CB0EEEB2258
:10624000113019F5F601EE0FFF1FEB5CFD4F1182C7
:10625000108285E1E82AE092DB0560EE75E08BEDC7
:1062600095E00E945704F601EE5CFD4F8091E20537
:10627000808362E0802F0E947D088B2D0E94001099
:10628000823008F4B8C112E0B7C1123051F4802F47
:106290008A5F0E940010682F802F0E94F70813E089
:1062A000ABC1133021F4882309F0A5C1A5C1143076
:1062B00051F4802F8A5F0E940010682F802F0E9467
:1062C000DA0815E099C1153089F4FF2009F494C16A
:1062D000802F0E94CF08F601EE0FFF1FEB5CFD4FF1
:1062E0008EE190E09183808316E086C11630A1F4A0
:1062F000F601EE0FFF1FEB5CFD4F80819181892B32
:1063000009F07AC1802F875F0E940010682F802FCC
:106310000E94F70817E070C11730D9F4FF2009F088
:106320006BC122E043E060E08E2D84610E94510544
:1063300020E040E060E08E2D8C610E945105802FAE
:10634000875F0E940010682F802F0E94DA0818E0F3
:1063500053C1183011F5FF2009F44EC1802F0E945F
:10636000CF088E2D8D618093DB0560EE75E08BED9F
:1063700095E00E9457042091E3054091E205609169
:10638000E1058E2D0E94510520E043E060E08E2D56
:1063900084610E94510519E02FC1193009F041C0F4
:1063A0008DE78093DB0560EE75E08BED95E00E9454
:1063B00057048091E00590E09601220F331F02C040
:1063C000959587952A95E2F780FF16C18B2D0E943F
:1063D0000010182F62E0802F0E947D08802F0E94FD
:1063E000CF0820E040E060E08E2D0E94510520E0C3
:1063F00040E060E08E2D82600E945105133039F03C
:106400008091240290912502892B09F473C0802F7A
:10641000875F0E940010682F802F0E94DA081AE020
:10642000EBC01A3061F4FF2009F4E6C020E040E040
:1064300060E08E2D8C610E9451051BE0DDC01B3099
:1064400009F05AC0FF2009F0D7C0802F0E94CF0862
:106450008E2D8D618093DB0560EE75E08BED95E010
:106460000E9457040E94A4302091E3054091E20568
:106470006091E1058E2D0E94510520E043E060E02F
:106480008E2D84610E9451051091E30510951093A3
:10649000E3050091E20500950093E205F090E10527
:1064A000F094F092E1050E94A4308091E305810F01
:1064B0008093E305882329F48091E2058F5F809320
:1064C000E2058091E205800F8093E205882329F49C
:1064D0008091E1058F5F8093E1056091E1056F0D8B
:1064E0006093E1052091E3054091E2058E2D8A61DC
:1064F0000E9451051EE080C01E3009F06EC08091E0
:10650000E00590E09601220F331F02C09595879514
:106510002A95E2F780FF70C062E0802F0E947D081C
:10652000802F0E94CF088B2D0E940010833031F005
:106530008091240290912502892B91F01092E00520
:106540001092E1051092E205F601EE0FFF1FEE0F2B
:10655000FF1FEA5DFD4F108211821282138203C079
:106560008E2D0E94B60A2091E3054091E2056091CC
:10657000E1058E2D0E9451051E2D12602091E3052C
:106580004091E2056091E105812F0E94510520E0D4
:1065900040E060E08E2D0E94510520E040E060E088
:1065A000812F0E945105F601EE5CFD4F20E04081F5
:1065B00060E08E2D84610E945105F601EE0FFF1FF1
:1065C000E35AF94F40815181662757FD6095762F38
:1065D0008E2D86600E9499080CC01F3069F4F60168
:1065E000EE5CFD4F22E0408160E08E2D84610E94D0
:1065F000510510E001C014E0EFEEF5E0CE0EDF1E15
:10660000F6011083DF91CF911F910F91FF90EF90D2
:10661000DF90CF90BF900895AC018091AB048823A8
:1066200019F480E090E008958BB78F7B8BBF909139
:106630003C0280913B02981711F490E01EC020911B
:106640003C02822F90E0FC0134E0EE0FFF1F3A95F0
:10665000E1F7E81BF90BDA01E559FC4F8FE00190F7
:106660000D928150E1F72F5F20933C0280913C0214
:10667000843111F410923C0291E08BB780648BBF9F
:10668000892F90E008950F931F93CF93DF93DA98AB
:1066900095E09093970480939804609399044093B5
:1066A0009A04C0E0D0E08E0109561B4FF8018081AA
:1066B0000E942310F80180832196C430D10599F7F8
:1066C000DA9ADF91CF911F910F910895EF92FF9287
:1066D0000F931F93CF93DF93DA9892E090939704F0
:1066E00080939804EE24FF24C62FD0E0229609C0A0
:1066F0008C0109561B4FF80180810E942310F8017C
:1067000080838E2D90E00894E11CF11C8C179D076E
:106710007CF3DA9ADF91CF911F910F91FF90EF9068
:1067200008950F931F93CF93DF93DA9892E090939D
:1067300097048093980460939904C0E0D0E08E01A0
:1067400009561B4FF80180810E942310F8018083B5
:106750002196C330D10599F7DA9ADF91CF911F9135
:106760000F910895EF92FF920F931F93CF93DF93B2
:10677000DA9893E09093970480939804EE24FF2492
:10678000C62FD0E0229609C08C0109561B4FF80194
:1067900080810E942310F80180838E2D90E0089460
:1067A000E11CF11C8C179D077CF3DA9ADF91CF91E5
:1067B0001F910F91FF90EF900895EF92FF920F932A
:1067C0001F93CF93DF93EC017A018B0110923E026D
:1067D00080913E0280933D0280913D0280933C0275
:1067E00080913C0280933B0264E88FE00E949133E9
:1067F00061E08EE00E94B233809199048F3F19F4DA
:106800001092AB049AC08091990487FFF1CF81E088
:106810008093AB04C130D10511F467E211C0C230DE
:10682000D10551F46FE08AE20E9491336FEB89E267
:106830000E94913367E038C0C330D10531F467E07E
:106840008AE20E9491336AEBF2CFC430D10511F491
:1068500063E0F6CFC530D10511F463E011C0C63056
:10686000D10551F463E08AE20E94913368E989E23C
:106870000E94913361E018C0C730D10551F460E047
:106880008AE20E94913368EB89E20E94913365E0CD
:106890000BC0289761F460E08AE20E94913360E9BE
:1068A00089E20E94913362E088E20E94913360E0C5
:1068B0008DE00E94913360E08CE00E949133D8011A
:1068C000C70143E0B695A795979587954A95D1F767
:1068D000809399048E2D8295880F807E80939A04F0
:1068E00010929B0410929C0464E080E00E94663346
:1068F0008FEF8093990480EE80939A0410929B040A
:1069000010929C0464E080E20E94663360E080E6BE
:106910000E94913361E18BE20E94913364E08FE049
:106920000E94913361E08EE00E94B233809199041D
:1069300087FDF8CF8BB780648BBFDF91CF911F911C
:106940000F91FF90EF900895AC018091AB048823E4
:1069500019F480E090E008958BB78F7B8BBF209176
:106960003D022F5F243109F420E080913E02281778
:1069700011F490E023C080913D0290E0FC0164E0BE
:10698000EE0FFF1F6A95E1F7E81BF90BE15CFD4F85
:10699000DA018FE00D9001928150E1F720933D02E2
:1069A00061E080E50E94B2338091990483FD05C0C7
:1069B00040E160E18CE20E94433391E08BB7806458
:1069C0008BBF892F90E008951F920F920FB60F9200
:1069D0001124EF92FF921F932F933F934F935F9356
:1069E0006F937F938F939F93AF93BF93CF93DF93D7
:1069F000EF93FF9361E08CE20E94B233809199049F
:106A0000E82E80FFC1C010913B021F5F143109F4D2
:106A100010E080913C02181709F4B1C090913B023C
:106A20008FE0989FE0011124C559DC4F6EE080E6AD
:106A30000E94B23380919B048695869586958170DD
:106A400089838981882309F45AC080919E048295A4
:106A50008695869581708A8380919B0490E0A0E062
:106A6000B0E0FBE1880F991FAA1FBB1FFA95D1F771
:106A70008B839C83AD83BE832B813C814D815E8162
:106A800080919C0490E0A0E0B0E0E3E1880F991FC2
:106A9000AA1FBB1FEA95D1F7822B932BA42BB52BF2
:106AA0008B839C83AD83BE832B813C814D815E8132
:106AB00080919D0490E0A0E0B0E0072E7BE0880F7D
:106AC000991FAA1FBB1F7A95D1F7702D822B932B8C
:106AD000A42BB52B8B839C83AD83BE832B813C8100
:106AE0004D815E8180919B0482958695877090E0B0
:106AF000A0E0B0E0822B932BA42BB52B0FC080918C
:106B0000990486958695869581708A8380919B04E9
:106B100082958695877090E0A0E0B0E08B839C839F
:106B2000AD83BE832B813C814D815E8180919A042F
:106B300090E063E0880F991F6A95E1F7AA2797FD17
:106B4000A095BA2F822B932BA42BB52B8B839C83E0
:106B5000AD83BE8380919E048F70888320E030E0F7
:106B6000F901E156FB4F8081F901EC0FFD1F87838E
:106B70002F5F3F4F2830310599F710933B0240E0DB
:106B800061E08CE20E944333E4FE96C040E060E1A5
:106B90008CE20E94433390913E0280913D0298170F
:106BA00009F48AC080913E029FE0899FE001112490
:106BB000C15CDD4F8F5F80933E028B819C81AD81F4
:106BC000BE8113E0B695A795979587951A95D1F74D
:106BD000809399048B819C81AD81BE818295880FC1
:106BE000807E80939A0489818823C9F180919A04D8
:106BF000886080939A0420919A048B819C81AD8156
:106C0000BE81FBE1B695A79597958795FA95D1F743
:106C10008370822B80939A0420919B048B819C81AA
:106C2000AD81BE81E3E1B695A79597958795EA95E5
:106C3000D1F7282B20939B0420919C048B819C816D
:106C4000AD81BE81072E7BE0B695A7959795879578
:106C50007A95D1F7702D282B20939C0404C01092B4
:106C60009B0410929C0488818F7080939D048A817C
:106C7000882329F080919D04806480939D0420E006
:106C800030E0F901EC0FFD1F8781F901E256FB4F5F
:106C900080832F5F3F4F2830310599F76DE081E504
:106CA0000E9466336BE080E50E94913380913E0242
:106CB000843111F410923E02FF91EF91DF91CF9158
:106CC000BF91AF919F918F917F916F915F914F9104
:106CD0003F912F911F91FF90EF900F900FBE0F905B
:106CE0001F901895823010F482E001C08E7F82B927
:106CF00085EC86BF85B3836085BB0895DC019091E8
:106D0000AC04961719F080E090E0089540E020E090
:106D100030E00BC0F901E155FB4F8081FD01E20F2E
:106D2000F31F80834F5F2F5F3F4F491799F71092F2
:106D3000AC0481E090E00895DC0140E020E030E028
:106D40000BC0FD01E20FF31F8081F901E854FB4FF6
:106D500080834F5F2F5F3F4F461799F76093AE04D4
:106D600008951F920F920FB60F9211248F939F9345
:106D7000EF93FF9381B1803629F485EC86BF1092A2
:106D8000AC0453C081B1803819F081B1883871F4F6
:106D900085EC86BF8091AC04E82FF0E093B1E1551B
:106DA000FB4F90838F5F8093AC043FC081B1803AEA
:106DB000D1F181B1882311F485ED36C081B1883AD3
:106DC000B1F41092AD049091AD04E92FF0E0E854D5
:106DD000FB4F808183B99F5F9093AD0485EC86BFA4
:106DE0009091AD048091AE049817F9F416C081B16A
:106DF000883BC9F49091AD04E92FF0E0E854FB4FD3
:106E0000808183B99F5F9093AD0485EC86BF90919C
:106E1000AD048091AE04981741F48091AD04815087
:106E20008093AD0402C085EC86BFFF91EF919F91E6
:106E30008F910F900FBE0F901F901895FF920F9398
:106E40001F93982F162F042FF22E8091C1048130AA
:106E500029F48BB78F7B8BBFAF980DC0823029F49C
:106E60008BB78F7B8BBFAE9806C0833021F48BB776
:106E70008F7B8BBFAD98892F0E942310812F0E949A
:106E80002310802F0E9423108F2D0E94231085B382
:106E9000806E85BB8BB780648BBF1F910F91FF9075
:106EA0000895CF93DF93CDB7DEB724970FB6F8944C
:106EB000DEBF0FBECDBF49835A836B837C83813095
:106EC00011F48AE005C0823011F48CE001C088E042
:106ED00029814A816B8181600E941E3724960FB6FA
:106EE000F894DEBF0FBECDBFDF91CF910895CF9351
:106EF000DF93CDB7DEB724970FB6F894DEBF0FBE91
:106F0000CDBF882311F4E0E005C0813011F4E2E048
:106F100001C0E4E0842F90E09695982F88279795FC
:106F20008795A0E0B0E09B0140E050E06CE0220FCC
:106F3000331F441F551F6A95D1F7822B932BA42B27
:106F4000B52B89839A83AB83BC8329814A816B816A
:106F50008E2F81600E941E3724960FB6F894DEBFF4
:106F60000FBECDBFDF91CF91089520E040E064E0F7
:106F700087E00E941E3720E040E060E281E10E944D
:106F80001E3720E040E060E089E00E941E3720E0EC
:106F900040E060E08BE00E941E3720E040E060E0CF
:106FA0008DE00E941E370895CF92DF92EF92FF92FC
:106FB0000F931F93CF93DF936C017B018091C104EA
:106FC000813029F48BB78F7B8BBFAF980DC0823097
:106FD00029F48BB78F7B8BBFAE9806C0833021F42A
:106FE0008BB78F7B8BBFAD98C0E0D0E087010C0FD3
:106FF0001D1FF601EC0FFD1F80810E942310F80178
:1070000080832196C430D10589F785B3806E85BB16
:107010008BB780648BBFDF91CF911F910F91FF9051
:10702000EF90DF90CF900895CF93DF93CDB7DEB789
:107030002C970FB6F894DEBF0FBECDBF813011F490
:107040008AE005C0823011F48CE001C088E08D83B5
:10705000BE016F5F7F4FCE0105960E94D4371C861C
:107060008A818B879B819A879C81998787FF03C040
:107070008FEF8C8701C01C8669857A858B859C85FE
:107080002C960FB6F894DEBF0FBECDBFDF91CF9127
:107090000895A0E0B0E0EFE4F8E30C945539EC017A
:1070A000688179818A819B816115710581059105CE
:1070B00049F484E2A82E89EDB82E8BE5C82E87E02E
:1070C000D82E02C05B016C01C601B5012DE133EF82
:1070D00041E050E00E94FC3827EA31E440E050E013
:1070E0000E94B6387B018C01C601B5012DE133EF5A
:1070F00041E050E00E94FC38CA01B90124E13BE0C4
:1071000040E050E00E94B638E61AF70A080B190B67
:1071100017FF08C08FEF9FEFAFEFBFE7E80EF91E34
:107120000A1F1B1FE882F9820A831B838FEF9FEFE0
:10713000AFEFBFE7E822F9220A231B23C801B701FA
:10714000EAE0CDB7DEB70C9471390E944938089552
:107150008FE091E00E944938089560930F01709389
:10716000100180931101909312010895629FD00144
:10717000739FF001829FE00DF11D649FE00DF11DF2
:10718000929FF00D839FF00D749FF00D659FF00DA1
:107190009927729FB00DE11DF91F639FB00DE11D8E
:1071A000F91FBD01CF0111240895AA1BBB1B51E19A
:1071B00007C0AA1FBB1FA617B70710F0A61BB70B67
:1071C000881F991F5A95A9F780959095BC01CD010C
:1071D000089597FB092E07260AD077FD04D0E5DF36
:1071E00006D000201AF4709561957F4F0895F6F748
:1071F000909581959F4F089597FB092E05260ED0F7
:1072000057FD04D014D00AD0001C38F45095409596
:10721000309521953F4F4F4F5F4F0895F6F790956A
:107220008095709561957F4F8F4F9F4F0895A1E294
:107230001A2EAA1BBB1BFD010DC0AA1FBB1FEE1FF0
:10724000FF1FA217B307E407F50720F0A21BB30B3B
:10725000E40BF50B661F771F881F991F1A9469F7B7
:1072600060957095809590959B01AC01BD01CF0113
:107270000895E199FECFBFBBAEBBE09A11960DB267
:107280000895E199FECFBFBBAEBB0DBA11960FB604
:10729000F894E29AE19A0FBE08952F923F924F928E
:1072A0005F926F927F928F929F92AF92BF92CF9296
:1072B000DF92EF92FF920F931F93CF93DF93CDB79F
:1072C000DEB7CA1BDB0B0FB6F894DEBF0FBECDBF17
:1072D00009942A88398848885F846E847D848C84E8
:1072E0009B84AA84B984C884DF80EE80FD800C81F1
:1072F0001B81AA81B981CE0FD11D0FB6F894DEBFD4
:0A7300000FBECDBFED010895FFCFD1
:10730A001414143C11DB249124AB1A3D2DF92529C0
:10731A002268219F20A41EF11CCC1BB51A611A7485
:10732A0028F8273E114011421144116913B0133550
:10733A00143E145A146D14741435197B1471180EF2
:10734A0018B21771254112D92780207E14B914C6A4
:10735A0014C714C914CB14CD14CF14D114D314D513
:10736A0014D714D914DB14DD14DF14E114E314E583
:10737A0014E714E914EB14ED14EF14F114F314F5F3
:10738A0014F7149E03A5039F03A003A103A203A35A
:10739A0003A403F914FC140C1510153C1735151128
:1073AA00173C15E816FE178C15A2154E16A61501E0
:0473BA0000000000CF
:00000001FF
